:100000000C948B040C94B3040C94B3040C94B304BC
:100010000C94B3040C94B3040C94B3040C94B30484
:100020000C94B3040C948C050C94AF280C945537A5
:100030000C94B3040C9412350C9450350C94B30406
:100040000C94B3040C94B3040C94B3040C94B30454
:100050000C94B30440202D202F2031203320352054
:1000600037203B203E204C20422044204620482080
:100070004A20CC24E624CF24D224D524DA24DC243C
:10008000E024E324E924E924D524D22497309A30CB
:100090009F30A430A730AA30AD30B330B830BF3075
:1000A000C430C730F330F730FC300131053109314D
:1000B0000F3115311A311E31243128310A320C32F8
:1000C0000E32123212321032163214320000000098
:1000D0000067582F00000000F567E630C8023200C4
:1000E0002F2CE80310093200802F2C0100000000A3
:1000F0000000000000000000000000000000000000
:100100002ECA7E3BC24CA40B0C49701700000000A5
:1001100043BFA80E0000000080D56610000000005C
:1001200080D0841F0000000031D561100000000065
:10013000C0D665100000000080D4651000000000EB
:1001400080D46510C60232002E2CE8030401320070
:10015000D2052C010006080001FF01010000010684
:10016000090001FF0302010002060A0001FF00006E
:10017000000006060E0000FF0302010005060D0048
:1001800000FF0203000004060C0000FF0302010050
:1001900003060B0000FF040600000706070000FF2F
:1001A00003020100B60D000E070F20205475726E79
:1001B0006967792034783600202020726373747662
:1001C0002E7275002020436865616C694368617216
:1001D00067657200202020207665723A20302E3329
:1001E0003200E60100006F7074696F6E73000100E9
:1001F00001000100010001000A0064000100030089
:1002000008000700070014000700010002000400B6
:1002100010004000000100046D5600206E6F007950
:10022000657300496E6600756E6C696D697465640E
:100230000063025E025902550250024B024602411F
:10024000024E695A6E004C69706F004C696C6F0009
:100250004C6966650050623F004E694D48004E692A
:10026000436400556E6B6E6F776E000098089808B7
:100270006C07102701980898086C0701000298087D
:1002800098086C070100039808DC006C070600045E
:10029000980898086C07030005980898086C0703ED
:1002A0000006980898086C07030007980898086CDF
:1002B00007030001000100010001000000B0041C60
:1002C00007520300000807B0044006E803000008D6
:1002D00007D0079209D60600000000E40C100ED0EB
:1002E00007E40C0000100E0410C409A60E000074F0
:1002F0000E6810B80B0A0F000040066C071405408A
:100300000600004E616D653A0045646974206E61B7
:100310006D653A0053034E03490344033F03310321
:100320002403000020202065646974206E616D65DF
:10033000002020637265617465206E616D650049FF
:10034000643A200049633A200043683A2000563A54
:100350002020004261743A20200025200046554CA0
:1003600020005245564552534520504F4C4152496A
:10037000545900706C656173652063616C696272C9
:10038000617465006265666F72652075736500460D
:10039000756E6374696F6E206E6F7400696D706C3A
:1003A000656D656E746564207965740064656C7450
:1003B0006120543D20006E6F742075736564005495
:1003C0006578743D0064656C746120563D20006D55
:1003D0006178566F75743D006E6F74207573656437
:1003E000006D6F6E69746F72206572726F72007249
:1003F0006561736F6E3A200070726F6772616D2075
:10040000636F6D706C657465002D00546578743D84
:10041000005662616C2E3D00566F7574203D0020C1
:100420006C696D69743D0056696E7075743D007736
:100430006972657320523D00626174742E20523DD2
:100440000020200062200074696D653A2020202081
:1004500020004C696D6974733A20006E2E612E0085
:1004600020202D2D20200043684342426C446946E1
:10047000435374534243684469437943594368443E
:100480006945420064542F6474002D645600562060
:100490006C696D69740087207B208B201D211821D9
:1004A000262181217C21C2212522F321F9215622F6
:1004B000E2226422000B0C0D64054305FF040000DA
:1004C0000708090A0D6405430516050C05FF04001D
:1004D0000000010203040D640555054D0543053771
:1004E00005FF040000000102030405060D64055524
:1004F000054D05430537052F052005FF0400006560
:10050000646974206261747465727900643E63206A
:100510006379636C6500633E64206379636C650096
:1005200073746F726167652B62616C616E630073D7
:10053000746F7261676500666173742063686172CD
:100540006765006469736368617267650062616C06
:10055000616E6365006368617267652B62616C61DF
:100560006E636500636861726765000106070500D8
:1005700002060708090B0C0D040503000206070814
:10058000090B0C0D0405030006070405000206070D
:1005900008090B0C0D04050300020F0B0C0D0405DC
:1005A0000300020A0E0F0B0C0D040503006578749E
:1005B0002054434F460063617020434F4646006914
:1005C0006E707574205600626174206469736300F4
:1005D000496F75743A20200076616C75653A200089
:1005E000436F6E6E65637420426174746572792125
:1005F0000008090A08090A11060806FF0500005646
:10060000623270696E3A200056623170696E3A202B
:100610000056623070696E3A2000270620060000FE
:1006200076616C75653A0074656D703A20003D0620
:1006300034060000706F696E7420322E00706F698E
:100640006E7420312E005F06520600005F065806C9
:1006500000003330306D4100313030306D410035B5
:10066000306D410006090A0B0C0D0E061E1F2021DD
:1006700022231200B806B206AC06A606A0069A0609
:1006800094068E0688060000566F75743A0056313F
:100690002D363A005662363A20005662353A20002E
:1006A0005662343A20005662333A20005662323A9B
:1006B00020005662313A200056696E3A2000080741
:1006C000FF06F306E706DB06CC06000065787065DA
:1006D00072742044414E474552210063616C696247
:1006E0002D3E554152540074656D702065787465D7
:1006F000726E0049206469736368617267650049BE
:100700002063686172676500766F6C74616765006D
:10071000300726071807000072657365742064654A
:100720006661756C740063616C6962726174650006
:1007300073657474696E67730080250000004B0058
:10074000000096000000E1000000C20100000070FF
:1007500017640007000C0005007800581B00000813
:100760000000000300432F6D0092078B0785077C74
:100770000773076578742E20416463006578742ED2
:1007800020646562006465627567006E6F726D61FA
:100790006C0064697361626C65640029081E081747
:1007A000080D080308F707ED07E207D907CF07C8C8
:1007B00007C007B70700002020207265736574002A
:1007C00073706565643A2000554152543A200062C6
:1007D000616C2E206572723A006469736368202B25
:1007E0003A00696E707574206C6F773A00636170BF
:1007F00020434F66663A00432F44206379636C655B
:10080000733A004E694364202D64563A004E694D98
:1008100048202D64563A0064542F64743A00657879
:1008200074726E2054434F3A00657874726E20548F
:100830003A2020200013161817190705061E1F203E
:1008400021222373200064200063200072657365F9
:1008500074696E6720656570726F6D3A00763A2034
:10086000372E312E32200000000000000000000072
:10087000000000000403000500000000000000006C
:100880000000000000000000000000000000000068
:100890000001000000204080000000000001020470
:1008A0000810204080000001020408102040800051
:1008B000000080402010080402010000010204082A
:1008C00010000202020000000000040404040404FA
:1008D00004040000030303030303030300000001F7
:1008E00001010101010101000002020202020000F7
:1008F000390036003300300000003B00380035007E
:10090000320000003A0037003400310079056E10E3
:100910004F202E25423611241FBECFE5D8E0DEBF82
:10092000CDBF10E0A0E6B0E0E4E0F3E702C0059040
:100930000D92A63EB107D9F714E0A6EEB0E001C0D3
:100940001D92A13AB107E1F719E0C6E1D9E004C070
:100950002297FE010E940739CC30D107C9F70E94C7
:10096000FE360C9480390C940000CF9388E20E94EC
:100970004A38C1E0892B09F0C0E089E20E944A3878
:10098000892B11F080E001C082E0C82B8AE20E942E
:100990004A38892B11F080E001C084E0C82B8BE23B
:1009A0000E944A38892B11F080E001C088E08C2B2E
:1009B000CF910895CF93C82F682F89E10E94DB372C
:1009C0006C2F8AE10E94DB376C2F80E20E94DB37BC
:1009D0006C2F89E00E94DB376C2F8BE00E94DB37A5
:1009E0006C2F80E1CF910C94DB3708958091FC004F
:1009F000882331F08091E6008F5F8093E60002C08B
:100A00001092E6008091FC008A3010F480E001C072
:100A100088E09091FC00943108F084E09091FC0013
:100A20009E3108F082E06091E60068238CE20C942D
:100A300014388093FC00089561E068278CE00C94E2
:100A4000143880E00E94523761E08CE00E94DB376E
:100A500061E08EE00E94DB3761E08EE10E94DB37CF
:100A600061E08CE20E94DB3761E08DE00E94DB37C1
:100A700061E08EE00E94DB3761E08FE00E94DB37AF
:100A800080E00E941C051092FC0020E042E060E142
:100A900087EE90E00E9486160E9477280E943723F6
:100AA0000E9497230E94FB050E94AE070C940E0D36
:100AB000CF93C82F682F617089E10E9414386C2F82
:100AC00062708AE10E9414386C2F647080E20E9488
:100AD00014386C2F687089E00E9414386C2F607194
:100AE0008BE00E9414386C2F607280E1CF910C94DF
:100AF0001438CF92EF920F9383E1C82E94E1E92E40
:100B000005E126E147E168E187EE90E00E943A17AF
:100B10000F91EF90CF9008951F920F920FB60F9202
:100B200011242F933F934F935F936F937F938F93F2
:100B30009F93AF93BF93EF93FF9320910001309168
:100B400001018091FE009091FF00820F931F90930E
:100B5000FF008093FE008091FE009091FF0026E050
:100B6000969587952A95E1F72091FE003091FF0038
:100B7000AC0166E0440F551F6A95E1F7241B350B65
:100B80003093FF002093FE002FB7F8943091FD00C2
:100B90003E3011F49BBD8ABD3091FD003D30A1F087
:100BA0002FBF0E94F604FF91EF91BF91AF919F91EB
:100BB0008F917F916F915F914F913F912F910F9006
:100BC0000FBE0F901F90189599BD88BDE9CF9FB7B4
:100BD000F89470930101609300018093FD008E30C2
:100BE00019F48FB5806804C08D3019F48FB5806218
:100BF0008FBD9FBF08951FBC80E18EBD2FB7F894B5
:100C000080E091E097BD86BD2FBF8EB5887F8EBDF9
:100C10008EB581608EBD89B7846089BF08958E309E
:100C200019F48FB58F7704C08D3019F48FB58F7D8F
:100C30008FBD08958091030190910401A091050159
:100C4000B0910601892F9A2FAB2FBB27A7FDBA952C
:100C5000089510920A01109209018617970768F407
:100C600080E090E4A0E0B0E0809303019093040161
:100C7000A0930501B093060108C0109203011092E1
:100C800004011092050110920601809103019091D8
:100C90000401A0910501B0910601BA2FA92F982F48
:100CA00088278093030190930401A0930501B093DA
:100CB000060181E0809302010895CF93DF93EC0158
:100CC000C13080E6D80770F4C13080E4D80760F402
:100CD0008EE00E940F0660E08EE00E941438BE0194
:100CE0008DE00CC0C0E0D0E68DE00E940F0661E010
:100CF0008DE00E941438BE0170548EE0DF91CF91D8
:100D00000C94E70590930A01809309016CEB76E659
:100D100080E00E94B00C9093080180930701089531
:100D2000CF93C82F882319F080E00E949D0661E0D0
:100D30006C278EE1CF910C941438CF93DF93C82F9A
:100D4000882319F080E00E9490068DE00E940F0633
:100D500060E08DE00E9414388EE00E940F0660E093
:100D60008EE00E9414381092020161E06C278FE03F
:100D70000E941438CC2361F080E00E948708EC01C7
:100D800086E00E948708BE01DF91CF910C9429066E
:100D9000DF91CF9108950F931F93809102018823D3
:100DA00009F474C080E00E949008209107013091FE
:100DB00008012817390730F480E00E949D06109240
:100DC000020164C082E00E949008409109015091A4
:100DD0000A0160E070E0009103011091040120918C
:100DE000050130910601481B590B61097109E4E0C6
:100DF000440F551F661F771FEA95D1F7040F151F83
:100E0000261F371F0093030110930401209305014F
:100E1000309306018091030190910401A091050196
:100E2000B0910601B7FF08C01092030110920401AF
:100E30001092050110920601809103019091040126
:100E4000A0910501B09106010197A046B10560F09F
:100E500080E090E0A0E6B0E080930301909304016D
:100E6000A0930501B09306018091030190910401C4
:100E7000A0910501B0910601892F9A2FAB2FBB27B6
:100E8000A7FDBA951F910F910C945D061F910F91CC
:100E90000895BC018EE00C94E7058770806287B9E5
:100EA0000895CF93DF9390916600891721F1809385
:100EB0006600C8B390E2899F90011124CF71C22BC4
:100EC00098B3E3EBF8E0E4912AB3DE2FD095D22378
:100ED0002AB38150823050F0892F8F71806C88BB8B
:100EE000E22BEABB8AE090E00E949F378FB7F8942C
:100EF000C8BBDABB8FBFDF91CF91089594B125B104
:100F000035E0839FF0011124EA5AFE4FE491F0E0AE
:100F1000EE0FFF1FEC54FE4F892F90E0922B918330
:100F20008083089510920B01E5E5F1E084910E9421
:100F30004D07E4E5F1E084910C945107369A089549
:100F40000E94FD229093D3018093D2010E944D23F1
:100F50009093D5018093D4010C947F0C60E08FE1D5
:100F60000E94143860E08FE10E94DB3761E081E08D
:100F70000E94DB3761E082E00E94DB3761E083E0C2
:100F80000E94DB3787E886B90C949207CF93DF93F2
:100F9000E0910B018E2F90E025E0E29FF0011124FB
:100FA000E85AFE4FE491EE2321F0C0913C02C1705B
:100FB00001C0C0E025E0289FF001299FF00D112419
:100FC000EC5AFE4F8491C11109C020915B0330910E
:100FD0005C03232B21F0873011F4C1E085E00E94EF
:100FE0005107E0910B01EF5F85E0E89FF0011124CC
:100FF000EB5AFE4F84910E944D078CE390E00E94D3
:101000009F370E949E073699FECFD0910B0181E059
:101010008D0F0E947E0725E0D29FF0011124EB5A2C
:10102000FE4F84910E944D078CE390E00E949F3711
:101030000E949E073699FECFC11104C080910B011A
:101040000E947E07E0910B01EF5F85E0E89FF001D1
:101050001124E95AFE4FE491E1110E94CB068091E0
:101060000B018E5F803118F480930B0102C0109247
:101070000B010E949908882341F080910B01811196
:1010800004C0DF91CF910C94A007DF91CF91089518
:101090000C949207CF93DF930E94820AC0912201A1
:1010A000D09123018091220190912301C817D90783
:1010B00019F40E94C607F6CFDF91CF910895CF9221
:1010C000DF92EF92FF92CF93DF93EC010E94D3283F
:1010D0006B017C01CC0EDD1EE11CF11C0E94C607D9
:1010E0000E94D3286C157D058E059F05B8F3DF910E
:1010F000CF91FF90EF90DF90CF900895E82FF0E030
:10110000EE0FFF1FEA52FE4F808191810895E82F74
:10111000F0E0EE0FFF1FE459FE4F808191810895AA
:10112000E82FF0E0EE0FFF1FEC54FE4F808191811D
:10113000089580913E0208958091220190912301AB
:101140000895E82FF0E0EE0FFF1FEC5DFE4F808169
:1011500091810895262F613110F4423040F021E052
:1011600030E0FC013383228331832083089550E0F3
:10117000BA01620F711D620F711D660F771F660F36
:10118000771F6E5F7F4F44E050E00C943B39282F6F
:10119000CA01213188F4623078F470E0620F711D69
:1011A000620F711D660F771F660F771F6E5F7F4F8F
:1011B00044E050E00C9459390895FF920F931F9327
:1011C000CF93DF9300D000D0CDB7DEB70CEC10E0AA
:1011D000F12CF801459155916591749149835A8399
:1011E0006B837C83AE014F5F5F4F60E08F2D0E9469
:1011F000C708F801349645915591659174914983DA
:101200005A836B837C83AE014F5F5F4F61E08F2D0C
:101210000E94C708F394085F1F4F81E1F812D9CFED
:101220000F900F900F900F90DF91CF911F910F9122
:10123000FF900895E82FF0E0EE0FFF1FE459FE4FF6
:1012400020813181EEEFE80FE53170F4F0E0ED58E8
:10125000FF4F8081882319F0813061F405C081E05F
:101260002333310540F404C081E0293E334018F4B3
:1012700080E0089581E00895CF93C0E08EE18C0F67
:101280000E941A09882329F0CF5FC630B9F786E09B
:1012900001C08C2FCF910895209198013091990130
:1012A00080910C0190910D01A0910E01B0910F0160
:1012B000820F931FA11DB11D80930C0190930D010E
:1012C000A0930E01B0930F01089560910C017091ED
:1012D0000D0180910E0190910F012DE730E040E06B
:1012E00050E00E94C438BB27A52F942F832F089568
:1012F0008091920190919301089580914A0190917B
:101300004B01039750F08091500190915101039748
:1013100020F083E090E00C943A0E80E0089590E095
:10132000880F991FFC01E459FE4F2081318162171B
:10133000730718F4261B370B04C0AB01421B530B79
:101340009A01FC01EC5DFE4F2730310518F0118247
:10135000108206C0208131812F5F3F4F318320836F
:10136000FC01E459FE4F718360830895AF92BF92F0
:10137000CF92DF92EF92FF920F931F93CF93DF9361
:101380001F92CDB7DEB700916C0110916D01609195
:101390007C0170917D0180917E0190917F016817A1
:1013A000790728F49C01261B370BB90102C0681B82
:1013B000790B8EE10E948F0960917E0170917F010F
:1013C00080918001909181016817790728F4FC01D0
:1013D000E61BF70BBF0102C0681B790B8FE10E946F
:1013E0008F0952E8E52E51E0F52E90E2F701619168
:1013F00071917F01892F99830E948F0999819F5F45
:101400009432A1F70E943C09F82E80E0A12CB12C67
:101410008F1569F0EEE1E80FF0E0EE0FFF1FE459E1
:10142000FE4F20813181A20EB31E8F5FF1CFB50137
:1014300082E10E948F09A114B10449F0A016B106FF
:1014400050F498012A193B09293E334020F05801F5
:1014500010E0F12C01C012E1B50183E10E948F0977
:101460006F2D70E085E10E948F09612F70E084E1AB
:101470000E948F090E9465098C010E943E238823E7
:1014800029F0E0907201F09073010BC00E94EE22EF
:10149000882329F0E0907001F090710102C0E12CE6
:1014A000F12CB70186E10E948F09B80188E10E9402
:1014B0008F099701D5010E94733830E1C32E37E2BE
:1014C000D32EE12CF12CA70196010E94C438B9015A
:1014D00087E10E948F099801D5010E947338A70106
:1014E00096010E94C438B90189E10F90DF91CF9134
:1014F0001F910F91FF90EF90DF90CF90BF90AF9032
:101500000C948F0910923D0210923C02E8EFF1E03A
:10151000119211921192119282E0EC33F807C1F707
:10152000089510921F0110921E0110921A0110923C
:101530001B0110921C0110921D01109216011092B5
:1015400017011092180110921901109221011092A6
:10155000200110921501109214010E94D32860936B
:10156000100170931101809312019093130108955B
:10157000E4E2F1E01192119281E0EC36F807D1F744
:1015800008950E94820A0C94B80A109223011092C6
:10159000220110920C0110920D0110920E01109276
:1015A0000F010E9448080E94C10A0E94910AECE6BD
:1015B000F1E01192119281E0E43BF807D1F7089530
:1015C00080913E0281110AC081E00E941C050E94A8
:1015D000C50A81E080933E020C944A080895109257
:1015E0003E0280E00C941C052091B6013091B701B9
:1015F0008091B4019091B5018217930718F4281BCC
:10160000390B02C020E030E081E0293E334008F48D
:1016100080E008958F929F92AF92BF92CF92DF9217
:10162000EF92FF92CF93DF93CDB7DEB728970FB637
:10163000F894DEBF0FBECDBFF82E5B0140E0682FEF
:10164000CE0105960E94AA0841E06F2DCE010196B9
:101650000E94AA082B813C8140E050E0CF80D884D2
:10166000E12CF12C2C193D094E095F09B50180E0F0
:1016700090E08D809E80A12CB12C681979098A098F
:101680009B090E94943829813A8140E050E0281952
:1016900039094A095B090E94E6382C0D3D1D4E1D93
:1016A0005F1D57FF03C020E030E0A901C901289663
:1016B0000FB6F894DEBF0FBECDBFDF91CF91FF9084
:1016C000EF90DF90CF90BF90AF909F908F90089554
:1016D0000F931F93CF93DF93C1E02091940130913A
:1016E000950180911A0190911B01A0911C01B0916C
:1016F0001D012231310531F0C0E02091B40130915B
:10170000B50104C02091920130919301820F931F83
:10171000A11DB11D80931A0190931B01A0931C0180
:10172000B0931D012091C2013091C3018091160137
:1017300090911701A0911801B0911901820F931F88
:10174000A11DB11D8093160190931701A09318015C
:10175000B093190180911E0190911F010196909301
:101760001F0180931E010E94D32800911001109147
:1017700011012091120130911301601B710B820B3A
:10178000930B61367A4E8105910508F479C08091FA
:1017900020019091210101969093210180932001D5
:1017A00020911E0130911F0140E050E060911A012C
:1017B00070911B0180911C0190911D010E94C43801
:1017C000890110921A0110921B0110921C011092B3
:1017D0001D01C11105C0B90180E00E940A0B8C01F6
:1017E000C091A201D091A3010C171D0720F0B801F0
:1017F0008BE10E948F09B8016C1B7D0B8AE10E946E
:101800008F0920911E0130911F0140E050E060914E
:1018100016017091170180911801909119010E9491
:10182000C4381092160110921701109218011092EC
:101830001901B90187E00E940A0B2091140130912F
:1018400015019093150180931401BC01621B730B69
:101850008CE10E948F0960911E0170911F018DE142
:101860000E948F0910921F0110921E010E94D3281E
:1018700060931001709311018093120190931301F2
:10188000DF91CF911F910F910895FF920F931F93B6
:10189000CF93DF9380912201909123010196909341
:1018A00023018093220108EF11E0C6EDD1E0F12C75
:1018B000F80161917191819191918F0120913C0288
:1018C00030913D0240E050E00E94C43829933993A2
:1018D000B9018F2D0E940A0BBC018F2D0E948F0928
:1018E000F394F1E1FF12E4CF0E94B6090E94C133E4
:1018F000DF91CF911F910F91FF900C94820ACF93AB
:10190000DF93E4EBF1E0C8EFD1E0219131918881E0
:101910009981AA81BB81820F931FA11DB11D89935B
:101920009993A993B99381E0E63DF80771F7809107
:101930003C0290913D02019690933D0280933C02BF
:101940000E94680B80913C0290913D028436910583
:1019500021F4DF91CF910C94450CDF91CF91089544
:101960008F929F92AF92BF92CF92DF92EF92FF92AF
:10197000CF93DF93CDB7DEB728970FB6F894DEBFCD
:101980000FBECDBFF82E5B0140E0682FCE0105965B
:101990000E94AA0841E06F2DCE0101960E94AA087C
:1019A00029813A8140E050E0CD80DE80E12CF12CAD
:1019B0002C193D094E095F09B50180E090E08F8048
:1019C0009884A12CB12C681979098A099B090E9475
:1019D00094382B813C8140E050E0281939094A09AC
:1019E0005B090E94E6382C0D3D1D4E1D5F1D57FF03
:1019F00003C020E030E0A901C90128960FB6F89491
:101A0000DEBF0FBECDBFDF91CF91FF90EF90DF9093
:101A1000CF90BF90AF909F908F9008950C94C50A7F
:101A2000462FE82FF0E0EE0FFF1FE459FE4F208114
:101A300031818250853130F4E82FF0E0ED58FF4FCE
:101A4000608101C061E0C9010C945B15825E0C9459
:101A5000870880916502089580916302811113C007
:101A60000E949908882381F00E949C0820913F02DF
:101A700030914002821B930B9C0181E0253031059F
:101A800018F080E0089581E008950F931F93CF939D
:101A9000DF9310E0CFEFDFEF00E0809165021817D1
:101AA00060F4812F0E94260D8C179D0710F0CE0147
:101AB00001C0012F1F5FEC01F0CF802FDF91CF918C
:101AC0001F910F910895CF93DF939091630291112D
:101AD00004C0DF91CF910C94260D90914902C82F3C
:101AE000D0E0992391F00E94260DCC0FDD1FFE015E
:101AF000E65BFD4FCA5ADD4F208131814881598113
:101B0000241B350B280F391F07C0FE01EE0FFF1FE6
:101B1000E65BFD4F20813181C901DF91CF910895AE
:101B2000CF93C82F80916302882341F0C11106C072
:101B30000E949C089093400280933F02C0936302EE
:101B40000E94D32860934102709342028093430223
:101B5000909344020E94B80A80916202811104C0ED
:101B60008C2FCF910C945805CF910895EF92FF924E
:101B70000F931F93CF93DF9381E00E94DA0485E1F6
:101B80000E9487088093650206E512E03AE4E32E9E
:101B900032E0F32EC0E0D0E08091650290E0C817FB
:101BA000D9076CF48C2F0E94260DF8018193919334
:101BB0008F01F701819391937F012196EDCF1092D0
:101BC00063021092620280E00E94900D1092400227
:101BD00010923F0210924102109242021092430270
:101BE00010924402DF91CF911F910F91FF90EF90DF
:101BF000089580E00E94900D81E080936202089534
:101C00000E94F90D80E00C94DA04FF920F931F9369
:101C1000CF93DF93809164020E94630DEC01F12C5D
:101C200001E010E080916502F816E8F48F2D0E9423
:101C3000630DAC0180916302802321F0C417D507A6
:101C400078F40DC02091590330915A032F5F3F4F14
:101C5000369527952C0F3D1F2417350708F4102BB8
:101C6000000FF394DFCF812FDF91CF911F910F9160
:101C7000FF9008951F93CF93DF93EC0110E08091C4
:101C80006502181748F48EE1810F0E94A1088C1795
:101C90009D0720F01F5FF3CF81E001C080E0DF915E
:101CA000CF911F910895BF92CF92DF92EF92FF9252
:101CB0000F931F93CF93DF938AE090E00E943A0E38
:101CC000882309F460C00E94450D809364020E943D
:101CD000260D8C0162E084E792E00E942919081722
:101CE000190748F17AE4E72E72E0F72EE6E5CE2EEA
:101CF000E2E0DE2EC0E0D0E0BB24B3948091650228
:101D000090E0C817D907CCF48C2F0E94260DF7015C
:101D1000819391937F01F601819391936F01801BD1
:101D2000910B2091590330915A032817390708F471
:101D3000B12C2196E3CFBB24B394109249020E94A8
:101D4000D328609345027093460280934702909394
:101D50004802BB2059F0DF91CF911F910F91FF9066
:101D6000EF90DF90CF90BF900C94F90D0E94050E7C
:101D7000DF91CF911F910F91FF90EF90DF90CF9067
:101D8000BF900C94900DDF91CF911F910F91FF9018
:101D9000EF90DF90CF90BF900895CF93809149024C
:101DA000811119C081E080934902809164020E94F0
:101DB000260DC0E080916502C81768F48C2F0E9440
:101DC000260DEC2FF0E0EE0FFF1FEA5AFD4F918336
:101DD0008083CF5FEFCFCF9108950F931F930E9421
:101DE000D32800914502109146022091470230917C
:101DF0004802601B710B820B930B28EE33E040E02E
:101E000050E00E94C438C9011F910F91089583E0EA
:101E100090E00E943A0E8823C9F0809163028111FC
:101E200003C00E94530E12C00E94CD0E0E94050EE8
:101E300090E0809590952091630230E08223932377
:101E4000892B81F40E94ED0E4F9760F40E942C0DB7
:101E5000882311F082E00895809162028823D1F3F3
:101E600081E0089580E00E94900DF0CF1F93CF9302
:101E7000DF93EC0110E080916502181780F4812F48
:101E80000E94260D8C179D0710F081E009C0812F5C
:101E90000E94630D8C179D07C0F71F5FECCF80E099
:101EA000DF91CF911F9108951F93CF93DF93EC01A2
:101EB00010E080916502181780F4812F0E94260D92
:101EC000C817D90710F081E009C0812F0E94630D67
:101ED000C817D907C0F71F5FECCF80E0DF91CF9123
:101EE0001F91089560916502662329F070E00E94B9
:101EF000B038CB01089580E090E008950E9402126E
:101F00000E944C1F85E00E944A310E94C32988E04C
:101F10000C944A310E9402120E94501F86E00E94D7
:101F20004A310E94C32988E00C944A31E09166024C
:101F3000F091670285919491FC010994E091660209
:101F4000F0916702329685919491FC010994E09199
:101F50006602F0916702349685919491FC01099490
:101F6000CF93DF931F92CDB7DEB7811107C00E94D8
:101F70002D1E0E949E0F0E948A0F0FC0813059F4BF
:101F800069830E942D1E0E949E0F6981611105C008
:101F90000E947E0F02C081E001C080E00F90DF91BF
:101FA000CF910895BF92CF92DF92EF92FF920F935D
:101FB0001F93CF93DF938C01C62E0E94960F0E9431
:101FC0000F1E0E94E8290E940212F12C82E0D82EF6
:101FD000C0E0D0E0EE24E3940E942F31811106C0CE
:101FE000F801EF0DF11D84910E941E200E949111B5
:101FF000B82E84E0B81209C0EF2DF0E03196E00F62
:10200000F11FE491E11123C005C082E0B81202C0C3
:10201000F110FA94EE2081F00E94F229D82E6C2D56
:102020000E94B00FE82E882339F00E949C08C81740
:10203000D90779F4E11003C0C11016C0E12C81E08A
:10204000B812CACF0E942D1E0E949E0F0DC0F3949D
:10205000E1CF0E949C08EC010E94A70FD82E6C2DA6
:102060000E94B00FE82EE6CF8D2DDF91CF911F910A
:102070000F91FF90EF90DF90CF90BF90089560E0B8
:1020800088E692E00E94701887FD0AC0811102C0A4
:102090000C94B42E992787FD909501970C94F02409
:1020A00008950E9421050E9434320E94F52E64EDAD
:1020B00071E084EC91E00E942F1F88EE93E00E9473
:1020C0005F0868EB71E08AEA91E00E942F1F88EEBA
:1020D00093E00E945F0880E00C94B23662EE71E0FB
:1020E00088E692E00E9482178CE890E09093690263
:1020F00080936802ECE6F2E08081805E8083089540
:10210000FC0124812052621710F40C947517862F5D
:1021100090E0821B91090E94F0196EE00C94441328
:10212000CF93DF93EC010E94FA118B819C810E9476
:1021300041130E94FE116A8188819981DF91CF91BC
:102140000C94D912FC0187818F3118F48F5F87833B
:10215000089586818F5F86830895FC018781882397
:1021600019F0815087830895868181508683089570
:102170000F931F93CF93DF93FC01C681D0E06D2FA7
:1021800080E00E94F41110E11C0F01E00C0F8C2F75
:102190000E949213011711F0C02FF7CFDF5FD230EA
:1021A00011F0C12FECCFDF91CF911F910F910895C6
:1021B0001F93CF93DF93EC0187EE90E00E946717A7
:1021C0001FEF8E81181721F0CE010E94B8101E81DA
:1021D0008F81682F70E094E0759567959A95E1F787
:1021E0008F700E94F4110E949111823049F0843066
:1021F00019F0813049F413C0CE010E94A210E1CF42
:10220000CE010E94AD10DDCF8830D9F68D81E881F6
:10221000F981E80FF11D8F819E81890F8083DF9105
:10222000CF911F910895FC017183608342833483B1
:102230002383158280E2868317820895CF93DF93EC
:10224000EC0187EE90E00E9467170E940212CE0117
:102250000E94901061E08D810E94F4110E94911102
:102260008230B1F0843041F08130C1F487EE90E0EB
:102270000E94601780E026C04D81242F30E08A81C3
:1022800090E00197281739072CF74F5F4D83E2CF75
:102290008D818823F9F281508D83DCCF8830D1F68F
:1022A00082E00E94E311823048F083E00E944A31CC
:1022B00087EE90E00E94601781E004C0CE010E948A
:1022C000D810C3CFDF91CF9108950C94B504E0915D
:1022D0007202F0E0EE0FFF1FE251FE4F85919491E4
:1022E0000895CF93DF93D82F0E94B504C82F8D1780
:1022F00041F082E390E00E945F080E94B504DC2F69
:10230000F5CF1092720210927102809373028823AB
:1023100019F080E00E94533180917302DF91CF91D8
:102320000895FF920F931F93CF93DF93C0E0D0E007
:10233000F12C0AEF10E040917202242F30E0220FBE
:10234000331FF901E65FFD4F65917491C8010E944A
:10235000B0386F5F7F4FC617D707A8F40E94B50447
:10236000F82E81E090E00E945F0880917302F816D9
:1023700041F08F2DDF91CF911F910F91FF900C9421
:1023800071112196D8CFFF20B1F0509171025F5F9B
:1023900050937102F901E450FE4F85919491252FDD
:1023A00030E02817390738F0463018F44F5F409373
:1023B00072021092710280917302DF91CF911F918E
:1023C0000F91FF900895CF93DF93D82FC0917302A0
:1023D0000E949111909172029D1711F08C17C1F318
:1023E000892FDF91CF910895462F682F87EE90E0D7
:1023F0000C94511660E080E00C94F41161E080E0F0
:102400000C94F41187EE90E00C944A16CF93DF936E
:10241000FC01DB018C91882389F0C081D181488344
:10242000808191810196918380838C9181508C93DE
:10243000882321F00190F081E02D1082DF91CF916F
:102440000895BF92CF92DF92EF92FF920F931F9366
:10245000CF93DF93EC018B017A014115510501F116
:10246000CA010E941439F8019081B82E981708F417
:10247000B92ECB2CD12CA601B701888199810E945D
:102480001D39288139812C0D3D1D39832883F801A0
:1024900080818B198083882319F0E881F98110826B
:1024A000DF91CF911F910F91FF90EF90DF90CF9030
:1024B000BF900895EF92FF921F93CF93DF9300D0C8
:1024C00000D0CDB7DEB77C01CA014B835C83698342
:1024D0007A830E944629182F69817A81DB018C91C9
:1024E0004B815C81811768F44FE3C7010F900F9017
:1024F0000F900F90DF91CF911F91FF90EF900C9470
:102500000612F70120813181210F311D3183208393
:10251000DB018C91811B8C93882321F00190F08149
:10252000E02D1082F9012AE030E0112369F0CA01A0
:10253000B9010E94B038405DBAE06B9F4019112488
:1025400042931150AB01F1CF0F900F900F900F906D
:10255000DF91CF911F91FF90EF9008950F931F93FC
:10256000CF93DF93CDB7DEB72B970FB6F894DEBFCE
:102570000FBECDBF8E010F5F1F4F1A87098727E05F
:102580002B87AC01BE01655F7F4FCE0109960E948B
:102590005A12B80187EE90E00E9449372B960FB689
:1025A000F894DEBF0FBECDBFDF91CF911F910F9189
:1025B00008950F931F93CF93DF93CDB7DEB7619745
:1025C0000FB6F894DEBF0FBECDBF0097D1F06131DA
:1025D00008F060E1062F10E0A801BC01CE010196D1
:1025E0000E942C39E1E0F0E0EC0FFD1FE00FF11F3D
:1025F0001082BE016F5F7F4F87EE90E00E944937E7
:1026000001C080E061960FB6F894DEBF0FBECDBF6B
:10261000DF91CF911F910F9108950F931F93CF9347
:10262000DF93CDB7DEB761970FB6F894DEBF0FBE6C
:10263000CDBF0097D1F0613108F060E1062F10E0C6
:10264000A801BC01CE0101960E941D39E1E0F0E035
:10265000EC0FFD1FE00FF11F1082BE016F5F7F4F77
:1026600087EE90E00E94493701C080E061960FB686
:10267000F894DEBF0FBECDBFDF91CF911F910F91B8
:10268000089560E10C940D13CF92DF92EF92FF92C8
:102690000F931F93CF93DF93CDB7DEB762970FB63B
:1026A000F894DEBF0FBECDBF009719F1613108F07D
:1026B00060E16C018E010F5F1F4F78018E2D801B32
:1026C000861768F4C6016A8B0E944B39F701819323
:1026D0007F01FFEFCF1ADF0A6A898111EFCFF8017E
:1026E000E60FF11D1082B80187EE90E00E94493795
:1026F00001C080E062960FB6F894DEBF0FBECDBF7A
:10270000DF91CF911F910F91FF90EF90DF90CF90CD
:102710000895882319F08FE192E002C08BE192E0E6
:102720000C944113682F87EE90E00C944B37CF93B5
:10273000DF93D82FC0E0CD1729F080E20E949213DA
:10274000CF5FF9CF8C2FDF91CF91089580E10C946A
:102750009713CF93DF931F92CDB7DEB7682F643006
:102760003CF080E269830E94921369816150F7CF47
:1027700083E292E00F90DF91CF910C940D136AE009
:102780000E94A43880E3890F0C949213DF92EF9299
:10279000FF920F931F93CF93DF93EC01F62ED42E6D
:1027A00016160CF086C068EE73E00E94B0388B01FC
:1027B000CB010E94462924E0E22EE80EEF142CF40F
:1027C00080E20E949213FA94F9CFFE14D4F0D11053
:1027D00018C0CE010E944629182FFA941F1524F420
:1027E00080E20E949213F9CFCE010E94AE128DE6D4
:1027F000DF91CF911F910F91FF90EF90DF900C949C
:1028000092132E2D332727FD3095245031094F2D5B
:10281000552747FD50954217530754F48F2DDF91EC
:10282000CF911F910F91FF90EF90DF900C94A9131F
:10283000C8010E94AE12CE0168EE73E00E94B0386B
:10284000EC011F2D1E1993E0F92EF10E84E0810F8B
:1028500018161CF48EE20E94921302E0010F1F145E
:1028600044F4CE0164E670E00E94B038862F0E94E6
:10287000BF13CE0164E670E00E94B038EC011F5F28
:1028800010163CF46AE070E00E94B038862F0E9477
:10289000BF13111674F4CE016AE070E00E94B038E4
:1028A000DF91CF911F910F91FF90EF90DF900C94EB
:1028B000BF13DF91CF911F910F91FF90EF90DF90A9
:1028C0000895EF92FF920F931F93CF93DF93EC0144
:1028D000F62E16160CF058C064E670E00E94B03870
:1028E0008B01CB010E94462933E0E32EE80EEF1462
:1028F0002CF480E20E949213FA94F9CF2E2D332704
:1029000027FD3095235031094F2D552747FD509510
:10291000421753074CF48F2DDF91CF911F910F91E8
:10292000FF90EF900C94A913C8010E94AE12CE0143
:1029300064E670E00E94B038EC010F2D0E1912E031
:10294000100F83E0800F18161CF48EE20E94921381
:10295000FF24F394F00E111644F4CE016AE070E007
:102960000E94B038862F0E94BF131F146CF4CE0152
:102970006AE070E00E94B038DF91CF911F910F9113
:10298000FF90EF900C94BF13DF91CF911F910F91A7
:10299000FF90EF900895BF92CF92DF92EF92FF9257
:1029A0000F931F93CF93DF938C01D62EB42EC22E9C
:1029B00016169CF52111DA94C8010E944629C82FE9
:1029C000D0E0ED2CFF24E7FCF094CE15DF052CF4CD
:1029D0008B2D0E949213DA94F4CFCC2019F08DE263
:1029E0000E949213EC16FD0664F48D2DDF91CF91B9
:1029F0001F910F91FF90EF90DF90CF90BF900C94BC
:102A0000A913C801DF91CF911F910F91FF90EF9013
:102A1000DF90CF90BF900C94AE12DF91CF911F91B9
:102A20000F91FF90EF90DF90CF90BF90089520E03E
:102A30000C94CB14CF93DF936CE370E00E94B0381A
:102A40009B01EC0140E363E0C9010E9417158AE392
:102A50000E94921340E362E0CE01DF91CF910C948B
:102A6000171540E20C941715292F221F2227221F29
:102A700019F091958195910940E20C94CB141616AA
:102A800034F461500E94611483E40C94921308950D
:102A9000161634F461500E94311585E20C9492139D
:102AA000089563303CF062500E94311588E192E055
:102AB0000C9441130895CF93DF93C62F141674F529
:102AC0006FEF640FC23081F030F4CC23B1F0C1302D
:102AD000B9F4D6E516C0C43061F068F0C53081F4B1
:102AE0000E94341585E516C0642FDF91CF910C94B8
:102AF0003F15D4EF03C06EEF640FD1E440E002C095
:102B0000D5E541E00E94C6138D2F0E949213C33079
:102B100029F488E6DF91CF910C949213DF91CF9145
:102B20000895462F63E00C945B15462F60E00C94EB
:102B30005B15462F61E00C945B15462F64E00C9406
:102B40005B15CF93DF93EC0160E08E810E94143817
:102B500081E090E00E949F3761E08E810E941438EE
:102B600081E090E00E949F3760E08E810E941438DF
:102B700084E690E0DF91CF910C949F37CF92DF9263
:102B8000EF92FF920F931F93CF93DF937C01C0E0EE
:102B9000D0E0C62ED12C87010C0F1D1F61E0F8017B
:102BA00087810E94DB37B6010C2E02C075956795B0
:102BB0000A94E2F76170F80187810E941438219627
:102BC000C430D10541F7C701DF91CF911F910F911B
:102BD000FF90EF90DF90CF900C94A115CF92DF92F1
:102BE000EF92FF920F931F93CF93DF937C01C0E08E
:102BF000D0E0C62ED12C87010C0F1D1F61E0F8011B
:102C000087810E94DB37B6010C2E02C0759567954F
:102C10000A94E2F76170F80187810E9414382196C6
:102C2000C830D10541F7C701DF91CF911F910F91B6
:102C3000FF90EF90DF90CF900C94A1151F93CF934E
:102C4000DF93EC01162F642F8C810E9414388D8144
:102C50008F3F19F060E00E9414388F85612F84FF48
:102C600006C0CE01DF91CF911F910C94EE1570E05C
:102C700084E0759567958A95E1F7CE010E94BE15AF
:102C8000612FCE01DF91CF911F910C94BE1540E0D2
:102C90000C941E1661E00E94471680ED97E00C949C
:102CA0009F37CF93DF93CDB7DEB728970FB6F89451
:102CB000DEBF0FBECDBF28E0EBE6F0E0DE011196EF
:102CC00001900D922A95E1F7FC012389421710F03B
:102CD0004FEF420FFE013196E40FF11DE40FF11D9D
:102CE0002081260F2068622F28960FB6F894DEBF49
:102CF0000FBECDBFDF91CF910C944716FC016089C8
:102D0000262F2460208B6C600C944716CF93DF93A2
:102D1000EC01423018F08F8588608F874B8B1C8ABE
:102D2000222329F0413019F48F8584608F8780E554
:102D300093EC0E949F3760E08C810E94143860E021
:102D40008E810E9414388D818F3F19F060E00E94BF
:102D500014386F8564FD1DC063E0CE010E94BE156E
:102D600084E991E10E949F3763E0CE010E94BE1585
:102D700084E991E10E949F3763E0CE010E94BE1575
:102D800086E990E00E949F3762E0CE010E94BE1566
:102D900016C06062CE010E94471684E991E10E944C
:102DA0009F376F856062CE010E94471686E990E0EA
:102DB0000E949F376F856062CE010E9447166F8523
:102DC0006062CE010E94471684E0888BCE010E948B
:102DD0007E16CE010E944A1682E0898B66E0CE0103
:102DE000DF91CF910C9447166F927F928F92AF92A2
:102DF000CF92EF920F931F93CF93DF93CDB7DEB7B0
:102E00003C01162F842F5D854E853F859889F301FF
:102E1000848325830683E782C086A18682865387C2
:102E200044873587968761E00E94DB37F30185810F
:102E30008F3F19F061E00E94DB3761E0F30186818A
:102E40000E94DB37112319F0F301178603C080E1DC
:102E5000F301878720E041E060E1C301DF91CF917A
:102E60001F910F91EF90CF90AF908F907F906F90C8
:102E70000C9486168F92AF92CF92EF920F93DC0153
:102E800013961C921E921297E2E9F0E0ED93FC93E8
:102E90001F921F921F921F928C2CAE2CC02EE22EDE
:102EA000042F2FEF462F61E00E94F4160F900F9031
:102EB0000F900F900F91EF90CF90AF908F9008955B
:102EC000FC0160896E7F608B68600C944716FC0182
:102ED0006089262F2160208B69600C94471641E0A1
:102EE0000E941E1681E090E00895FC0127818085F4
:102EF000E22FF82FE60FF11DE60FF11D8591949159
:102F00000C9441130F931F93CF93DF93EC018B012C
:102F1000CB010E940029682FCE010E94E5178AE9A3
:102F200090E09983888318870F83DF91CF911F9159
:102F30000F910895DF92EF92FF920F931F93CF931B
:102F4000DF93EC01F62E69871A8681E08D8382E09B
:102F5000D82EEE24E3948E01075F1F4F0E9491113B
:102F6000482F823011F0843061F4E881F9810280C9
:102F7000F381E02D6F2DCE010995F986DA86ED8279
:102F800004C0813089F0883079F0C8010E94D729C7
:102F90008111ED828D81882319F0CE010E941218D3
:102FA0008A858F5F8A87DACF8FEF898781E08E836A
:102FB0008D83483009F080E0DF91CF911F910F9110
:102FC000FF90EF90DF9008950895FC0180EA90E073
:102FD0009183808312821382648381E08583868358
:102FE0000895FC012281211103C081E082830895AC
:102FF000438130E0240F311D848190E00197281730
:10300000390714F44F5F43830895FC0182818823BC
:1030100019F08150828308958381882311F08150B3
:10302000838308951F93CF93DF93EC0110E0612F0A
:1030300080E00E94F41180E20E949213E881F981FD
:103040006B81610F0190F081E02DCE0109950E9406
:10305000A6131F5F123059F76A8180E00E94F411B5
:103060008EE30E9492136A818FE00E94F4118CE338
:103070000E9492131D82DF91CF911F9108950F93AB
:103080001F93CF93DF93EC010E949111182F0E94A0
:103090002F31882321F081E08D838FE71CC00B81C5
:1030A0008A81080F123031F0143039F4CE010E94B9
:1030B000051803C0CE010E94F1178B819A81890FF8
:1030C000081711F081E08D838D81882319F0CE01DE
:1030D0000E941218812FDF91CF911F910F910895B7
:1030E000EF92FF921F93CF93DF931F92CDB7DEB77E
:1030F0007C0181E0F701858311E0C70169830E94AB
:103100003F186981811102C0F7011682F70196818B
:10311000911108C0883031F481E0868383819281E7
:10312000890F09C0662311F0F7011583813029F753
:103130009111E3CF8FEF0F90DF91CF911F91FF900F
:10314000EF9008950F931F93CF93DF93EC018B01C2
:1031500050E00E945A124AE3B801CE01DF91CF91AC
:103160001F910F910C940612EF92FF920F931F93F1
:10317000CF93DF9300D01F92CDB7DEB78C01462FDF
:1031800009969A8389838EE08B83D801EC91F0E0D5
:10319000EE0FFF1FEF5CFD4FE590F490BE016D5FF9
:1031A0007F4FCE0101960E94A218A701BE016D5F5C
:1031B0007F4FCE0101960E94211240E2BE016D5F59
:1031C0007F4FCE0101960E940612F8014181528183
:1031D000BE016D5F7F4FCE0101960E945A124FE2F1
:1031E000BE016D5F7F4FCE0101960E940612D8018D
:1031F00017964D915C911897BE016D5F7F4FCE0180
:1032000001960E945A120F900F900F90DF91CF916C
:103210001F910F91FF90EF90089527E1289FB00133
:10322000299F700D112464577F4F47E150E084E7D8
:1032300092E00C943B3927E1289FB001299F700D43
:10324000112464577F4F47E150E084E792E00C94EB
:103250005939DC01EC91B5E0EB9FF0011124E60F48
:10326000F11DEE0FFF1FED54FD4F859194910895D0
:10327000DC01EC9145E0E49FF0011124E60FF11D23
:10328000EE0FFF1FED54FD4F8591949117962D91F0
:103290003C911897AC01429FC001439F900D529FF3
:1032A000900D11240895FC01A181B2812091530356
:1032B000309154030E94733824E630E040E050E03F
:1032C0000E94C438293EFDEF3F074105510520F01B
:1032D00028EE3DEF40E050E0C9010895FC01208157
:1032E000213029F420914F033091500309C022303E
:1032F00029F420914D0330914E0302C020E030E0CC
:10330000FC0187819085AC01249FC001259F900D11
:10331000349F900D1124089580914B0390914C039C
:103320000895FC016081F9E06F9FB0011124655997
:103330007D4F49E050E00C940B39DC01EC91F0E05A
:10334000EE0FFF1FEF5CFD4F859194910C940D13D0
:1033500060E170E00C949D19CF93DF93EC018881BC
:1033600060E0811108C0CE010E94381967E00E9418
:10337000991587E011C0CE010E94381965E00E94BE
:1033800099158FE20E9492138F8198850E94AE1248
:1033900083E40E94921388E0DF91CF91089566E064
:1033A000FC01838194810E94951586E0089566E072
:1033B000FC01858196810E94951586E00895FC01A7
:1033C00081819281883EFDEF9F0729F487E292E098
:1033D0000E94411303C067E00E94911588E00895A0
:1033E00027E1AC01249FC001259F900D11248B562D
:1033F0009F4F08950F931F93CF93DF93CDB7DEB701
:10340000A4970FB6F894DEBF0FBECDBF8C01AB0101
:10341000BC01CE0101960E945C1BCE0101960E9468
:10342000CA1B87E1FE013C96D80101900D928A9556
:10343000E1F7A4960FB6F894DEBF0FBECDBFDF91C3
:10344000CF911F910F910895FC012081260F283004
:1034500010F4208302C0FC0110820C94911961E0E9
:103460000E9438199C0140E050E060E870EF8AEF5C
:1034700092E00E94C438213787E1380741055105A1
:1034800020F020E737E140E050E0C901089561E015
:103490000E9438199C0140E050E060E47BE48CE439
:1034A00090E00E94C438213D87E03807410551056E
:1034B00020F020ED37E040E050E0C90108950F937F
:1034C0001F93CF93DF9300D0CDB7DEB78C01698314
:1034D0007A830E942F1AAC0169817A81C801039610
:1034E0000F900F90DF91CF911F910F910C9476293F
:1034F0000F931F93CF93DF9300D0CDB7DEB78C012E
:1035000069837A830E94471AAC0169817A81C80174
:1035100005960F900F90DF91CF911F910F910C9412
:103520007629DC01EC91BAE0EB9FF0011124EB5419
:10353000FD4F6591749184ED92E60E94B038CB0105
:1035400008950F931F93CF93DF9300D0CDB7DEB7CD
:103550008C0169837A830E94911AAC0169817A8116
:10356000C80107960F900F90DF91CF911F910F9197
:103570000C947629CF93DF93EC010E94911A2F814E
:1035800038858217930710F498878F83CE010E94A5
:103590002F1A2B813C818217930710F49C838B8315
:1035A000CE010E94471A2D813E818217930710F4A5
:1035B0009E838D83DF91CF910895CF93DF93EC01AC
:1035C00048EE5DEF01960E94762989819A819C835D
:1035D0008B832881233039F49C01369527953695C5
:1035E00027953C832B839E838D83CE01DF91CF91E2
:1035F0000C94BA1ADF92EF92FF920F931F93CF931E
:10360000DF9300D01F92CDB7DEB749E050E061EA0A
:1036100072E084E792E00E940B3984E792E00E9416
:10362000BA1A00E010E05EE0D52E6DE7E62E62E00B
:10363000F62EDB82FA82E98241E0400FBE016D5F27
:103640007F4FCE0101960E94A218C8010E941B194B
:103650000F5F1F4F0032110561F70F900F900F9011
:10366000DF91CF911F910F91FF90EF90DF90089520
:10367000262F443019F06FEF7FEF02C061E070E059
:10368000223089F028F4222341F0213049F00895B6
:10369000233061F0243069F008950B960C94241ABD
:1036A0000B960C94A11A0B960C94DD1A0B960C94A5
:1036B0005F1A0B960C94781AEF92FF920F931F9358
:1036C000CF93DF93EC018B017A0164E173E00E94F8
:1036D00082178FEF898786EA90E09983888387E154
:1036E000F801DE011B9601900D928A95E1F7FBA28D
:1036F000EAA2DF91CF911F910F91FF90EF90089573
:103700000F931F93CF93DF93CDB7DEB728970FB6F4
:10371000F894DEBF0FBECDBF8C01BC016C5E7F4F45
:1037200029E033E04EE050E0CE0101960E941311F3
:10373000CE0101960E941E1181E0F8018583289632
:103740000FB6F894DEBF0FBECDBFDF91CF911F91B2
:103750000F910895CF93DF93EC016AA17BA16F5F76
:103760007F4F0B960E94B4180E9402120E94FA1119
:1037700083E093E00E9441130E94FE116EE0CE01AF
:1037800044960E94D9120E94C32983E0DF91CF9111
:103790000C944A31DF92EF92FF920F931F93CF93D5
:1037A000DF93CDB7DEB767970FB6F894DEBF0FBED5
:1037B000CDBF8C0187E1D82EC8010B967C0160E05B
:1037C000C8010E94701887FD2AC0853031F086300C
:1037D00041F4C8010E94801BF2CFC8010E94AA1BBD
:1037E000EECFF701DE0111969D2D01900D929A9575
:1037F000E1F7682FC8010E949A17811109C0FE01E4
:103800003196D7018D2D01900D928A95E1F7D7CF92
:1038100083E00E944A31C7010E94BA1AD0CF67964E
:103820000FB6F894DEBF0FBECDBFDF91CF911F91D1
:103830000F91FF90EF90DF9008951F93CF93DF9348
:10384000EC01162F0E947517CE0109960E94CC2913
:10385000882311F0298501C02FEF332727FD3095EC
:10386000812F90E02817390719F11230C1F048F480
:10387000112381F01130E1F4CE010B960E94AC19B6
:1038800017C0133089F0143099F4CE010B960E94C2
:10389000D7190EC0CE010B960E94A81909C0CE01FF
:1038A0000B960E94DF1904C0CE010B960E94CF191F
:1038B00080E0DF91CF911F910895CF93DF9300D0E7
:1038C000CDB7DEB789839A830E94FA1189819A81E4
:1038D0000E9441130E94FE118091D4029091D50262
:1038E0000E941439892B51F08FEE93E00E9441130E
:1038F0008091D4029091D5020E9441130F900F90B5
:10390000DF91CF910C94A6138091470390914803C7
:10391000892BA1F08CE10E94870865E02AE0AC01C8
:10392000249FC001259F900D11240E9434158DE61F
:103930000E94921383E40E94921304C088ED93E0E6
:103940000E9441130C94A6138AE10E94870865E047
:103950000E9434158DE60E94921386E50E94921310
:103960000C94A61390E0880F991F62E089599B4F31
:103970000C940D130F931F93CF93DF9361E084E7B3
:1039800092E00E9438198C0162E084E792E00E9484
:103990003819EC0183E10E9487088017910790F4A1
:1039A000C817D90788F49C012C1B3D0BC8018C1B40
:1039B0009D0B64E670E00E94B038C9010E94B038E7
:1039C000862F03C084E601C080E0DF91CF911F9174
:1039D0000F910895613011F40C94630D0C948326BB
:1039E000CF93DF93D82FC62F8EE18D0F0E941A0937
:1039F000882351F06C2F8D2F0E94EA1C46E06C2F1B
:103A0000DF91CF910C945B1580E694E0DF91CF912C
:103A10000C9441130F931F93CF93DF93C82F162F4E
:103A20000E94FA110E942C0D811108C083E090E0E1
:103A30000E943A0E882341F080E209C08091490239
:103A4000882321F082E403C08DE601C082E60E9453
:103A50009213809163028823C9F0D0E001E0809145
:103A60006402D81731F080916302802321F081E352
:103A700003C08FE501C080E30E949213000FDF5F57
:103A8000D63069F780E20E94921303C087E00E945B
:103A90009713D1E0DC0F8D2F0E94BF138AE30E94A1
:103AA0009213C11108C00E943E23882321F00E9476
:103AB0004D23892B29F5612F8C2F0E94F01C0E9429
:103AC000A6130E94FE1102E00C0F802F0E94BF136C
:103AD0008AE30E949213612F8D2F0E94F01C83E0D5
:103AE0008C0F0E94BF138AE30E949213612F802FD4
:103AF0000E94F01CDF91CF911F910F910C94A6139F
:103B00008BE594E00E944113DACF88E10E94870898
:103B100068E00E94911580E20C9492130E94FA11C1
:103B200084E792E00E94531968E00E94911580E2B8
:103B30000E9492130E946C2667E00E9495150E94D5
:103B4000A6130E94FE1182E594E00E94411367E0F3
:103B500080913703909138030E9499150C94A61315
:103B60000F931F9360919602709197028091980233
:103B70009091990220918B02222371F00E94D32808
:103B8000009196021091970220919802309199022B
:103B9000601B710B820B930B28EE33E040E050E08A
:103BA0000E94C438C9011F910F9108950E94EE220E
:103BB000811110C00E943E23882331F00E94EE2222
:103BC00081110AC084E40BC00E942C0D811106C033
:103BD0008EE405C083E403C085E401C082E40E9452
:103BE000921380E20E9492130E94B01D0E941A1547
:103BF00080E20C9492130E94FA110E94851D67E0E6
:103C000086E10E94100D0E94A6130E94FE110E94E0
:103C1000D61D67E083E10E94100D0C94A6130E944C
:103C2000D3286093960270939702809398029093A2
:103C300099021092920210929302109294021092A2
:103C4000950210928E0210928F02109290021092A2
:103C5000910281E080938B0208950F931F930E943D
:103C6000D3280091960210919702209198023091EA
:103C70009902601B710B820B930B609396027093F9
:103C80009702809398029093990210928B021F9151
:103C90000F9108950E94F42281111DC00E944423B7
:103CA000811119C00E942C0D882351F1809192023C
:103CB00090919302A0919402B091950280599F4FE8
:103CC000AF4FBF4F8093920290939302A0939402C0
:103CD000B0939502089580918E0290918F02A091E9
:103CE0009002B091910280599F4FAF4FBF4F809388
:103CF0008E0290938F02A0939002B0939102D2CF44
:103D00000895CF92DF92EF92FF920E94FA1187E41A
:103D100094E00E9441130E94B01D0E941A150E9457
:103D2000FE1184E494E00E9441136091920270912C
:103D30009302809194029091950238EEC32E33E065
:103D4000D32EE12CF12CA70196010E94C438C901A1
:103D50000E941A1581E494E00E94411360918E0242
:103D600070918F028091900290919102A70196012B
:103D70000E94C438C901FF90EF90DF90CF900C945F
:103D80001A150E94FA1188E394E00E9441130E94E0
:103D90008D2668E00E949D150E94A6130E94FE11C8
:103DA00082E10E941A09882349F08FE294E00E9480
:103DB00041130E94932668E00E949D150C94A6135F
:103DC0000E94FA1187E294E00E94411367E086E0C6
:103DD0000E94100D0E94A6130E94FE118FE194E034
:103DE0000E94411347E061E0809155039091560392
:103DF0000E945B150C94A6130E94FA1188E194E0CE
:103E00000E94411367E080E00E94100D0E94A613FB
:103E10000E94FE1181E194E00E94411367E082E17B
:103E20000E94100D0C94A6130E94FA118BE094E0EE
:103E30000E9441138091470390914803892B29F0F8
:103E400065E087E00E94100D04C089E094E00E94C4
:103E500041130E94A6130E94FE110C94A6130F9307
:103E60001F93CF93DF9300D0CDB7DEB78B0189834B
:103E70009A830E9402120E94FA1189819A810E94FB
:103E800041130E94FE11C8010F900F90DF91CF9156
:103E90001F910F910C94411388EF93E00C945D1CDB
:103EA00081EE93E00C945D1C0E94FA110E94851D26
:103EB0000E94841C0E94FE110E94D61D0C94A41C1A
:103EC0000E94FA118FEC93E00E94411367E08BE1AE
:103ED0000E94100D0E94A6130E94FE1185EC93E033
:103EE0000E9441130C94A41C0E94FA118FEB93E0E2
:103EF0000E9441138091470390914803892B41F020
:103F000069E080911401909115010E943F1504C051
:103F100086EB93E00E9441130E94A6130E94FE11BB
:103F20008CEA93E00E9441130C94841C6CE973E0CA
:103F30008FE893E00C942F1F0E94961F0C94C329C6
:103F400064E873E083E793E00E942F1F88E893E121
:103F50000C94E3280E94FA1182E693E00C9441133A
:103F6000CF930E94FA1164E070E084E792E00E942F
:103F70009D1980E20E94921384E792E00E94AC199E
:103F800080E20E9492138091D6020E94B21C0E948D
:103F9000FE110E94BA1C90E08436910569F48CE809
:103FA00092E00E94CC29882321F084E00E9497139C
:103FB0000AC08DE593E005C062E00E9431158AE5F4
:103FC00093E00E9441138CE892E00E94CC29882360
:103FD00019F0C0918C0201C0CFEFC0FF05C065E0B1
:103FE00080E00E94100D03C085E00E94971380E2DC
:103FF0000E9492138091740284508430A8F4C1FF0F
:1040000005C065E082E10E94100D03C085E00E94BA
:104010009713C2FF05C00E943C09CF910C94BF13B7
:1040200080E2CF910C94921366E08091750290919A
:1040300076020E949115CF910C94A61390918D0257
:104040009F5F90938D0290E0FC013197EF30F10576
:1040500028F5E65DFF4F0C9405390C94FB1D0C947C
:104060008E1D0C94811E0C94141F61E005C061E04C
:1040700083E00C940A1D64E080E0FBCF64E0F8CF9D
:104080000C94B01F0C94C11E0C94FC1E0C94E01EEA
:104090000C94601F0C94741F0C94541F08958FEFA0
:1040A00080938C0208950F931F93CF93DF930E9408
:1040B0001623C0917702D091780261E084E792E004
:1040C0000E9438198C01CE0165E070E00E94B03882
:1040D0008FE00E94B00CEC0140E0BC01C8010E94DE
:1040E000B7268FE00E94CB26CE01DF91CF911F91A2
:1040F0000F910C94022381E00C9424230E947D09EB
:10410000882321F00E94FD220C94722708951092BA
:104110009A020C945320CF93DF930E947E200E943A
:104120007809EC0180919A02811111C062E084E764
:1041300092E00E9438198C179D0748F481E0809323
:104140009A0280917702909178020E9410230E9437
:104150007D09882381F064E084E792E00E943819A9
:104160008C179D0740F48EE894E09093D5028093DD
:10417000D40281E02EC0809120019091210102970C
:1041800038F180919B02882389F08AE10E94870898
:10419000EC0184E792E00E946E19D195C195D10996
:1041A0008C179D071CF48AE894E0DFCF80919C0275
:1041B000882371F08CE10E948708EC0184E792E08B
:1041C0000E948C198C179D071CF484E894E0CDCFD5
:1041D00082E0DF91CF91089580939C0260939B02CF
:1041E00008957093A00260939F0290939E02809323
:1041F0009D0208950F931F93CF93DF93C0919D026B
:10420000D0919E02CE010E94720F8C010E9478090B
:10421000C817D90738F4C801DF91CF911F910F91CA
:104220000C94540F81E0DF91CF911F910F9108956D
:1042300081E00E9484230C94000E0E9476230E9449
:10424000B60D1092A10280E10C94CB260F931F9320
:10425000CF93DF930E94FA20182F0E944D23EC0188
:104260000E947D09882311F001E001C0012F809197
:10427000A102882329F0BE01812F0E94232701C0BB
:10428000812F882329F081E00E94842381E00CC0E3
:10429000002349F0BE01812F0E943F288C179D0703
:1042A00011F00E94692382E0DF91CF911F910F915D
:1042B0000895BC0180E10E94B00C0C945B260F9322
:1042C0001F93CF93DF938C01EB010E94F120BE017D
:1042D00080E10E94B00C40E0BC01C8010E94B726FA
:1042E000CE016AE070E00E94B038CB01DF91CF913F
:1042F0001F910F910C94592181E00E9424230C946A
:10430000000E0E94B60D0E9416238FE00C94CB265F
:104310000F931F93CF93DF931F92CDB7DEB78C011E
:104320008FE049830E94B00C4981BC01C8010F9005
:10433000DF91CF911F910F910C94B726BC018FE0B4
:104340000E94B00C0C945B260F931F93CF93DF93C6
:10435000C0913703D0913803CE010E94720F8C01B7
:104360000E9478098C179D0738F4C801DF91CF911E
:104370001F910F910C94360F81E0DF91CF911F9127
:104380000F9108951F93CF93DF930E94A421182FBC
:104390000E94FD22EC01BC01812F0E94232788236B
:1043A00029F081E00E94242381E019C00E947D0948
:1043B000811107C0111105C0CE010E947426882307
:1043C00069F00E942C0D811109C0BE01812F0E944D
:1043D0003F288C179D0711F00E94022382E0DF9195
:1043E000CF911F9108950E947C210E9418210C9466
:1043F000000ECF93DF931F92CDB7DEB79091A3024B
:10440000913039F018F0923039F00FC00E94C2217B
:104410000CC00E94262109C00E94070F823089F03B
:1044200089830E94F32189810CC0813051F49091DD
:10443000A202992331F082E08093A3020E94B60D7C
:1044400082E00F90DF91CF9108950E94B60D809188
:10445000A4029091A5020E94720F0E94540F88231B
:1044600029F00E9481211092A30208950E941D212B
:1044700081E08093A1028093A30208958093A20219
:1044800008950F931F93CF93DF93EC018A019093CC
:10449000A5028093A40240E00E948821B801CE01C9
:1044A000DF91CF911F910F910C945F210E94762391
:1044B00087E080938C0282E080938D020E944331DA
:1044C00083E08093A7020895FF920F931F93CF93E9
:1044D000DF9380E00E941A0901E008278091A6027C
:1044E000882381F00E943C0990917B02FF24F39481
:1044F000981301C0F12C11E0811110E0913021F4EA
:10450000112311F010E0F12C82E10E941A09882396
:10451000A9F082E10E948708EC0180E00E948708F0
:10452000C817D90728F49C012C1B3D0BE90102C0D8
:10453000C81BD90BC53FD14008F001E0F11002C003
:1045400087E001C083E080938C02112329F08091E1
:104550008C02825080938C02002329F080918C027F
:10456000815080938C02F11004C0111102C000230D
:1045700011F081E001C088E00E944A310E9465117B
:10458000811102C01092A702F11008C0111106C0DB
:10459000011104C00E946511883041F08091A7028A
:1045A000823011F481E008C082E006C08091A70249
:1045B0008F5F8093A702F2CFDF91CF911F910F9170
:1045C000FF90089581E00E9484238FEF80938C02F6
:1045D00088E00C944A318093A602089581E090917E
:1045E000AA02911180E0089581E02091A802309103
:1045F000A902232B09F480E008958091A8029091EC
:10460000A9020895813B20E3920710F080EB90E32C
:104610009093A9028093A8020E9482060C94C10A7A
:10462000BC018FE00E94B00C0C9402238091AA027E
:10463000882349F080E090E00E94022381E00E94FC
:104640009D061092AA020895CF93C82F8091AA02C6
:1046500081110BC0CC2349F080E090E00E9402233E
:1046600080E00E949D06C093AA02CF91089580E049
:1046700090E00E94022381E00C94242381E0909139
:10468000AF02911180E0089581E02091AD02309158
:10469000AE02232B09F480E008958091AD02909141
:1046A000AE020895482F8091AB029091AC02209108
:1046B000AD023091AE028217930711F4442341F00A
:1046C0009093AE028093AD020E9449070C94C10AF8
:1046D0000895813020E4920710F080E090E49093F8
:1046E000AC028093AB0281E00C9452238091AF0224
:1046F000882349F080E090E00E94692381E00E94D5
:1047000090061092AF020895CF93C82F8091AF0208
:1047100081110BC0CC2349F080E090E00E94692316
:1047200080E00E949006C093AF02CF91089580E090
:1047300090E00E94692381E00C9484230895809185
:104740007402873051F09CEF980F943048F08150FC
:10475000823048F482EC92E0089589EB92E008956B
:104760008BEC92E0089580EB92E008958EEA94E05D
:10477000909367028093660290917402945081E056
:10478000943008F080E00E94EB2261E08BE695E037
:104790000E94D20F91E0813009F090E0892F0895B6
:1047A0000F931F93CF93DF930E943E2200917902D3
:1047B00010917A02C0917702D091780263E084E789
:1047C00092E00E943819A801BE010E94412288EAA5
:1047D00094E0909367028093660260E080E795E042
:1047E000DF91CF911F910F910C94D20FEF92FF9216
:1047F0000F931F93CF93DF938C01C7E7D2E0E8803C
:10480000F98061E084E792E00E94381940E0B70146
:104810000E94882188819981B8010E94B038CB011B
:104820000E949E2182EA94E0909367028093660240
:1048300060E08DE895E0DF91CF911F910F91FF909F
:10484000EF900C94D20FCF93DF93C0917702D09169
:10485000780261E084E792E00E94381941E0BE01ED
:104860000E94882182EA94E0909367028093660216
:1048700060E08DE895E0DF91CF910C94D20F81E05C
:104880002091470330914803232B09F480E061E035
:104890000E94EC2086E994E0909367028093660280
:1048A00060E082EA95E00C94D20F62E084E792E047
:1048B0000E9438196091790270917A02E0917B022E
:1048C000F0917C024091570350915803E49F90016E
:1048D000E59F300DF49F300D1124820F931F0E942D
:1048E0005F218CE994E0909367028093660260E018
:1048F0008CE795E00C94D20FCF93DF93C0917902AF
:10490000D0917A0262E084E792E00E943819BE01F9
:104910000E945F218CE994E0909367028093660285
:1049200060E089E995E0DF91CF910C94D20F84EAA1
:1049300091E0909367028093660260E088E895E0DA
:104940000C94D20FCF93C82F8093D60224EB34E07F
:104950003093D5022093D4028D3030F4E82FF0E06C
:10496000E655FF4F808101C080E0809367000E9480
:104970008F320E94E00A0E94B623882361F184E00E
:104980000E944A318C2F90E08D30910510F5FC018A
:10499000E75CFF4F0C9405398AE090E008C00E9464
:1049A000972419C00E94552416C085E090E00E940B
:1049B000F62311C080E001C081E00E94D0230BC02B
:1049C0000E943F2408C00E947C2405C00E9423242A
:1049D00002C00E949C1F0E94EF0ACF910C946C347D
:1049E0000F931F93CF93DF93EC010E940D190E9448
:1049F0009F238C0160E0C8010E94701887FD29C0C8
:104A000090917402E82FFF27E7FDF095973019F495
:104A1000EF52FB4F0FC08CEF890F843018F4EB512D
:104A2000FB4F08C09150923018F4E054FB4F02C085
:104A3000EB54FB4F84918D3049F4BE0184E792E042
:104A40000E94FA19CE010E941B19D1CF0E94A22404
:104A5000D1CFDF91CF911F910F9108956DEE74E04A
:104A60008BEC92E00E94821765EC74E082EC92E09D
:104A70000E94821767ED74E089EB92E00E94821732
:104A800068EB74E080EB92E00C948217FC014281A9
:104A900053814115510591F0A081B181B7FF03C049
:104AA000B195A195B10928EE33E00E9482389A01B0
:104AB00040E050E00E94C438C901089580E090E0D1
:104AC00008950F931F93CF93DF9300D000D0CDB7FD
:104AD000DEB78C01862FF801628173810E940A0B78
:104AE0009C838B83F801808191819A838983CE0195
:104AF00001960E9446250F900F900F900F90DF9126
:104B0000CF911F910F9108950F93FC01CB010023CA
:104B100041F04617570708F4CA016417750748F4AF
:104B200007C06417750708F4CA014617570708F449
:104B3000BA019783868391838083138212821582C0
:104B4000148233872287681B790B718760870F91E6
:104B50000895FC019B0140E050E086819781281B6D
:104B6000390B41095109A285B3850E9489382085F6
:104B70003185442737FD4095542F0E94E638211592
:104B8000310581E04807510524F457FD05C0C901EE
:104B900008958FEF9FEF089580E090E00895DF92F1
:104BA000EF92FF920F931F93CF93DF93EC012A8133
:104BB0003B812417350720F4FA01E21BF30B03C0F5
:104BC000F901E41BF50B8C819D81969587958E17D5
:104BD0009F0770F5888199818617970720F4FB015C
:104BE000E81BF90B03C0FC01E61BF70BEF2B01F1EF
:104BF0002417350738F48A01021B130B7B01E81ACE
:104C0000F90A06C07C01E61AF70A8901041B150B94
:104C1000C7010E941929D82E888599850E941929D3
:104C2000D81206C01D830C83F986E8861B870A8785
:104C3000DF91CF911F910F91FF90EF90DF9008953A
:104C40000F931F93CF93DF93EC018B019A01A885FB
:104C5000B9850E9482382A853B8540E050E00E9459
:104C6000E638C801A0E0B0E082179307A407B507B3
:104C70001CF41F821E8204C0021B130B1F830E83B1
:104C8000DF91CF911F910F910895EF92FF920F93B3
:104C90001F93CF93DF93EC018B017A010E94CF2504
:104CA000A701B801CE01DF91CF911F910F91FF9025
:104CB000EF900C94202690933E0380933D0308953B
:104CC0008091D902813029F480913D0390913E0377
:104CD000089580E090E008956091390370913A035F
:104CE0008091DB020C940A0B2091DE02213041F00E
:104CF00041E020913D0330913E038217930708F075
:104D000040E0842F08952CE0829FC001112460911F
:104D1000DB0289519D4F0C9461256091DB028FE28B
:104D200093E00C946125CF93DF9300D000D0CDB7F2
:104D3000DEB780E00E9487089A83898382E10E941F
:104D4000870829813A81281B390B3A83298386E118
:104D50000E9487089C838B83CE0101960E94462582
:104D60000F900F900F900F90DF91CF910895909337
:104D700038038093370370933A0360933903CB0170
:104D80006AE070E00E94B03870933E0360933D0388
:104D90004093DA020895EF92FF920F931F93CF93FF
:104DA000DF9391E09093D902FF24F3948F3009F0C0
:104DB000F12C8093DB0268EC70E00E94B00C9093C1
:104DC0003C0380933B030E94780920913D0330917E
:104DD0003E0340913703509138030F2DBC0187E209
:104DE00093E00E9484250E94290D8093DC0280912B
:104DF0003703909138030E94720FEC0110E08CE0B1
:104E0000E82E8091DC02181798F4812F0E94630D20
:104E1000BC0120913D0330913E03E19EC00111246D
:104E20000F2DAE0181529D4F0E9484251F5FE9CF57
:104E30001092DE021092DD02DF91CF911F910F914F
:104E4000FF90EF9008950F931F93CF93DF93082F58
:104E5000EB018091DA028823C9F040913B03509125
:104E60003C0320913D0330913E032417350708F49D
:104E70009A012C173D0710F4109262028091DE0215
:104E8000813021F00E94070F8093D9028091D902CE
:104E9000813011F58091DE02823041F411E02091E1
:104EA0003D0330913E03C217D30708F010E00E9483
:104EB00060268C179D0770F0111102C0002351F07D
:104EC0009091DD0281E0890F8093DD0281E09A30CC
:104ED00020F402C01092DD0280E0DF91CF911F919B
:104EE0000F9108950F931F93CF93DF93EC010E94CE
:104EF0007809AE01BC0187E293E00E94452610E0EC
:104F00000CE08091DC02181770F4812F0E94630D71
:104F1000BC01019FC0011124AE0181529D4F0E942E
:104F200045261F5FEECFDF91CF911F910F9108951E
:104F3000CF92DF92EF92FF920F931F93CF93DF9365
:104F4000609137037091380387E293E00E94A925AE
:104F50008C0180913703909138030E94720F7C017D
:104F6000D12C9CE0C92E8091DC02D81698F4CD9CFF
:104F7000E0011124C152DD4FB701CE010E94A925E5
:104F80000817190728F0B701CE010E94A9258C0146
:104F9000D394E9CFC801DF91CF911F910F91FF907A
:104FA000EF90DF90CF9008950F931F93CF93DF93EF
:104FB000EB018093350390933603209139033091B0
:104FC0003A038C012817390708F489010E946026EA
:104FD0008017910708F4C801C817D90711F120916B
:104FE000DE022230A9F48C179D0790F020913D033A
:104FF00030913E032C173D07A0F0409133035091B0
:10500000340320913F02309140024217530749F088
:1050100020913F02309140023093340320933303B8
:1050200001C0CE01DF91CF911F910F9108950F9391
:105030001F93CF93DF93EC010E947809909328038C
:1050400080932703D0932A03C093290310E00CE038
:105050008091DC02181770F4812F0E94630D019F6C
:10506000F0011124E152FD4F91838083D383C283E9
:105070001F5FEECFDF91CF911F910F9108951F9386
:10508000CF93DF93182FEB01CB010E947227CE0143
:105090000E9417280E9498279093D8028093D702E5
:1050A000BE010E94D4272091DE02211110C01123DD
:1050B00089F08091DA02882321F00E94F90D109284
:1050C000620281E08093DE0280E090E003C022E093
:1050D0002093DE02DF91CF911F91089560913F03ED
:1050E000709140038091410390914203089512BE54
:1050F0008DE78CBF88E083BF83B7836083BF89B7A8
:10510000826089BF089580913F0390914003A091F0
:105110004103B09142030196A11DB11D80933F034D
:1051200090934003A0934103B093420308950E94DB
:1051300083280E941B320E94E6290E94F504809178
:105140006800815019F080936800089581EE809383
:1051500068000E949E230E944C090C944A1E1F92D4
:105160000F920FB60F9211242F933F934F935F939B
:105170006F937F938F939F93AF93BF93EF93FF931F
:105180000E949728FF91EF91BF91AF919F918F91CE
:105190007F916F915F914F913F912F910F900FBE33
:1051A0000F901F9018952FB7F89460913F0370915E
:1051B000400380914103909142032FBF96958795BC
:1051C000779567950895CF92DF92EF92FF92CF93F4
:1051D000DF93EC010E94D3286B017C01CC0EDD1E15
:1051E000E11CF11C0E94D3286C157D058E059F05DE
:1051F000C8F3DF91CF91FF90EF90DF90CF900895AB
:1052000040E0FC01259134910296232B11F04F5F71
:10521000F8CF842F0895282F81E090E03AE02150C4
:1052200038F0AC01349FC001359F900D1124F7CFA9
:10523000089597FD02C081E008958FEF0895CF9201
:10524000DF92EF92FF92CF93611571058105910571
:1052500021F461E070E080E090E0C0E02AE0C22E3E
:10526000D12CE12CF12CCF5FA70196010E94C4380C
:10527000CA01B9012115310541055105A1F78C2F4E
:10528000CF91FF90EF90DF90CF900895BC0180E028
:1052900090E00C941F29FC0120813181260F371FDB
:1052A00037FF03C011821082089550E04217530760
:1052B0001CF4518340830895318320830895FC01B9
:1052C00020813181260F371F121613062CF081E042
:1052D00090E091838083089550E0421753071CF4B7
:1052E000518340830895318320830895DF92EF92A4
:1052F000FF920F931F93CF93DF93EC018A01DD247C
:10530000D394161617060CF0D12CE880F980B7015B
:1053100080E090E00E941F29823028F082500E9495
:105320000B299C0102C021E030E0C701B9010E94B5
:10533000B038009739F0DD2019F0281B390B04C074
:105340009C010FC0DD2069F0C801821B930BE81699
:10535000F90618F42E0D3F1D01C0980139832883EA
:105360000AC02E153F0518F4E21AF30A02C0E12C18
:10537000F12CF982E882DF91CF911F910F91FF907C
:10538000EF90DF9008950E9491118111FCCF0E944F
:1053900091118823E1F30895FC01208127FD05C0C8
:1053A000818186958F5F8170089580E00895FC016A
:1053B000208127FD09C081819FEF980F9695282FA6
:1053C000269581E0921301C080E008950895089524
:1053D0006CE87EE680E00E94B00C909344038093DA
:1053E00043030895CF93DF9380E00E9490082091BB
:1053F0004303309144032817390718F487EC95E0EC
:1054000012C086E00E948708EC0186E00E941A091B
:10541000882379F08091550390915603C817D907D6
:1054200040F48FEB95E09093D5028093D40280E016
:105430002BC088E10E948708EC0184E792E00E947B
:105440005319883E2DEF920731F08C179D0718F401
:1054500086EB95E014C08091470390914803892B17
:1054600011F482E011C087E00E948708209149036F
:1054700030914A0328173907A0F78DEA95E09093F9
:10548000D5028093D40281E0DF91CF9108950F93EC
:105490001F93CF93DF938C01443019F0CFEFDFEFF0
:1054A00002C0C1E0D0E00E946711D8011B96EC91C8
:1054B000F0E0EE0FFF1FE459FE4F9C01C29FC001B8
:1054C000C39F900DD29F900D112420813181820FB6
:1054D000931F91838083DF91CF911F910F91089546
:1054E000EF92FF920F931F93CF93DF931F92CDB74D
:1054F000DEB78C01443021F0EE24EA94FE2C03C088
:10550000EE24E394F12C69830E946711D8011B9665
:10551000ED91FC911C976981E60FF11DE491F0E09B
:10552000EE0FFF1FE459FE4F9C01E29EC001E39E77
:10553000900DF29E900D112420813181280F391F8A
:10554000318320830F90DF91CF911F910F91FF90B6
:10555000EF900895CF93DF9300D000D0CDB7DEB7A2
:1055600080E00E947E089A83898382E10E948708F6
:105570009C838B83AE014F5F5F4F61E080E00E94B0
:10558000C7080F900F900F900F90DF91CF91089563
:105590000F931F93CF93DF93CDB7DEB728970FB646
:1055A000F894DEBF0FBECDBF8C0189E00E947E085B
:1055B0009E838D8388E00E948708800F911F9887C3
:1055C0008F838AE00E947E089A8389830F811885E1
:1055D0008FE10E948708800F911F9C838B83AE010F
:1055E0004B5F5F4F61E089E00E94C708AE014F5FEB
:1055F0005F4F61E08AE00E94C70828960FB6F894D2
:10560000DEBF0FBECDBFDF91CF911F910F910895E7
:105610000F931F93CF93DF9300D000D0CDB7DEB7A9
:105620008C018AE00E947E089A83898389E00E9427
:105630008708800F911F9C838B83AE014F5F5F4F64
:1056400061E08AE00E94C7080F900F900F900F90C2
:10565000DF91CF911F910F91089560E070E080EE8F
:1056600095E00E942F1F80E00E941A09811106C058
:105670000E9491118130B9F780E0089581E008958A
:10568000CF93DF9300D000D0CDB7DEB7962F5A83EB
:1056900049833C832B838E3121F4C9010E94C82A9F
:1056A0000DC08F3121F4C9010E94082B07C0AE0143
:1056B0004F5F5F4F61E0892F0E94C7080F900F90E6
:1056C0000F900F90DF91CF910895FF920F931F934A
:1056D000CF93DF93F62E142F022F83E00E944A31DE
:1056E000812F0E948708EC0181E080933E020E9496
:1056F0004A08802F0E947E08AC019E01602F812FF6
:105700000E94402B0E944A08FF2039F0DF91CF9180
:105710001F910F91FF900C94AA2ADF91CF911F91B6
:105720000F91FF900895EF92FF920F931F93CF93E5
:10573000DF93CDB7DEB72E970FB6F894DEBF0FBE5E
:10574000CDBF0E9476230E942D2B882309F43FC0F1
:1057500067EF75E0CE0101960E9482178FEF8A876E
:105760008BEB90E09A83898384EF95E09D878C870B
:1057700086E08E8761E0CE0101960E947018F82EB7
:1057800087FD25C0082F112707FD1095F801EC5063
:10579000FA4FE4908E2D0E941A09882359F30E9433
:1057A0004A0810923E026F2DCE0101960E949A1770
:1057B000882349F0F801EF50FA4F24914E2D60E014
:1057C0008F2D0E94652B81E080933E02D3CF81E034
:1057D0000E9484232E960FB6F894DEBF0FBECDBF75
:1057E000DF91CF911F910F91FF90EF900895EF926D
:1057F000FF920F931F93CF93DF93CDB7DEB72E9712
:105800000FB6F894DEBF0FBECDBF0E9476230E9474
:105810002D2B882359F164E776E0CE0101960E9492
:1058200082178FEF8A878BEB90E09A8389838BE6D0
:1058300096E09D878C8789E08E8761E0CE01019696
:105840000E947018F82E87FD11C0082F112707FD40
:105850001095F801E559F94FE49086E08F156CF347
:105860008E2D0E941A09882341F310C081E00E9406
:1058700084232E960FB6F894DEBF0FBECDBFDF9106
:10588000CF911F910F91FF90EF9008950E944A08C9
:1058900010923E026F2DCE0101960E949A17882326
:1058A00049F0F801EC59F94F24914E2D61E08F2D0C
:1058B0000E94652B81E080933E02BFCF0E94FA11C7
:1058C00088ED95E00E94411365E080914503909139
:1058D00046030E9431150E94A6130E94FE1180ED1E
:1058E00095E00E94411367E086E10E94100D0C9440
:1058F000A613EF92FF920F931F93CF93DF93082F7E
:105900001092460310924503811105C00E94162390
:10591000CCE2DCE004C00E947623CAEADAE00E940E
:105920002D2B811102C0C0E04AC0F12C6AE0E62EA6
:105930000E945E2C0E949111182F0E9467119C01F9
:10594000E29EC001E39E900D1124143079F4409141
:105950004503509146034C175D0750F79C01240FF7
:10596000351F30934603209345030FC01230C1F416
:10597000409145035091460348175907C8F2481B08
:10598000590B5093460340934503809145039091F2
:105990004603011103C00E94022302C00E94692332
:1059A000183021F4FF2021F2C1E009C0111103C019
:1059B000FF24F394BDCF113009F0BACFB4CF81E00A
:1059C000011103C00E94242302C00E9484238C2F53
:1059D000DF91CF911F910F91FF90EF900895DF928B
:1059E000EF92FF920F931F93CF93DF9300D000D0DD
:1059F000CDB7DEB7162F7A01D22E0E94792C8823DC
:105A0000E9F083E00E944A31FC82EB828D2D0E94F6
:105A10007E089A838983AE014F5F5F4F612F8D2D82
:105A20000E94C708802F0E947E089A838983AE0156
:105A30004F5F5F4F612F802F0E94C7080F900F901C
:105A40000F900F90DF91CF911F910F91FF90EF90EA
:105A5000DF9008950F93CF93DF93CDB7DEB72997EB
:105A60000FB6F894DEBF0FBECDBF6CE476E0CE017A
:105A700001960E94821760E0CE0101960E94701884
:105A800087FD0EC0811103C042E350E002C048EE22
:105A900053E00FE022E0682F80E00E94EF2CEBCF74
:105AA00029960FB6F894DEBF0FBECDBFDF91CF9120
:105AB0000F9108950F93CF93DF93CDB7DEB729975A
:105AC0000FB6F894DEBF0FBECDBF66E476E0CE0120
:105AD00001960E94821760E0CE0101960E94701824
:105AE00087FD0EC0811103C042E350E002C04CE2CA
:105AF00051E000E123E0682F81E00E94EF2CEBCF22
:105B000029960FB6F894DEBF0FBECDBFDF91CF91BF
:105B10000F9108951F93CF93DF9300D000D01F9271
:105B2000CDB7DEB7182F6D830E947E089A838983D4
:105B3000812F0E9487089C838B83AE014F5F5F4F4C
:105B40006D81812F0E94C7080F900F900F900F90CA
:105B50000F90DF91CF911F9108950F931F93CF93D3
:105B6000DF93CDB7DEB72C970FB6F894DEBF0FBE2C
:105B7000CDBF182F062F6AE176E0CE0101960E9474
:105B800082178FEF8A8723EC30E03A8329831C87C2
:105B900061E0CE0101960E94701887FD13C081114B
:105BA000F7CF10923E0260E0CE0101960E949A1754
:105BB000882321F0602F812F0E948A2D81E080931D
:105BC0003E02E6CF2C960FB6F894DEBF0FBECDBFD7
:105BD000DF91CF911F910F9108951F93CF93DF9382
:105BE000CDB7DEB729970FB6F894DEBF0FBECDBF95
:105BF000182F6EE276E0CE0101960E94821760E0D7
:105C0000CE0101960E947018682F87FD04C0812F75
:105C10000E94AD2DF4CF29960FB6F894DEBF0FBECB
:105C2000CDBFDF91CF911F910895CF93DF93CDB773
:105C3000DEB72A970FB6F894DEBF0FBECDBF82E065
:105C4000809367006EEB76E0CE0101960E9482178A
:105C500060E0CE0101960E94701887FD29C08A87F6
:105C60000E948F320E94E00A8A85823099F03CF4CB
:105C7000882369F08130B9F40E942A2D14C0843041
:105C800081F05CF0853079F40E94932B0CC00E9467
:105C9000F72B09C00E945A2D06C087E00E94ED2D07
:105CA00002C00E9476340E94EF0A0E946C34D0CF6A
:105CB00083E0809367002A960FB6F894DEBF0FBE8C
:105CC000CDBFDF91CF9108951F93CF93DF93EC0168
:105CD000162F0E947517CE0109960E94CC298823A1
:105CE00011F0898501C08FEF992787FD9095612F6D
:105CF00070E08617970741F0EB85FC85E60FF71FEC
:105D000084916D850E94100DDF91CF911F910895B0
:105D10001F93CF93DF93EC01162F0E947517CE01CE
:105D200009960E94CC29882311F0298501C02FEF04
:105D3000332727FD3095812F90E02817390769F028
:105D4000111105C067E08B850E94100D06C08B8580
:105D50000E947E0867E00E943115DF91CF911F916C
:105D6000089581E00C94B236CF93DF93CDB7DEB7C0
:105D700029970FB6F894DEBF0FBECDBF60E177E084
:105D8000CE0101960E94821760E0CE0101960E942A
:105D90007018813049F0823051F081110BC087E4D6
:105DA00093E00E94222FF0CF0E94152EEDCF0E948B
:105DB000B12EEACF87FFE8CF29960FB6F894DEBF61
:105DC0000FBECDBFDF91CF910895DC015696ED91C6
:105DD000FC915797EE0FFF1FEE0FFF1FE75CF84F88
:105DE0006591759185919491089548E150E06EE632
:105DF00073E087E493E00E943B390C94E72948E183
:105E000050E06EE673E087E493E00E9459390C9409
:105E1000E72948E150E06DE477E00C940B3987E422
:105E200093E00E94092F0C94FF2EFC0122853385FC
:105E30002630310520F025E030E0338722870895B1
:105E40000C94E7290F931F93CF93DF93CDB7DEB761
:105E5000A3970FB6F894DEBF0FBECDBF8C01BC0177
:105E6000CE0101960E944F2FCE0101960E946C2F09
:105E700088E1FE013C96D80101900D928A95E1F7E8
:105E80000E94FF2E0E94E729A3960FB6F894DEBF6A
:105E90000FBECDBFDF91CF911F910F9108950F934A
:105EA0001F93CF93DF93EC018B016BE977E00E94A6
:105EB00082178FEF89878BEC90E09983888388E144
:105EC000F801DE011B9601900D928A95E1F7DF91B2
:105ED000CF911F910F910895DF92EF92FF920F9350
:105EE0001F93CF93DF93CDB7DEB768970FB6F894C3
:105EF000DEBF0FBECDBF7C018C01055F1F4F88E167
:105F0000D82E60E0C7010E94701887FD2AC08D302E
:105F100039F4C8010E94092F83E00E944A31F1CF71
:105F2000F801DE0111969D2D01900D929A95E1F7F1
:105F3000682FC7010E949A17811109C0FE0131968E
:105F4000D8018D2D01900D928A95E1F706C083E06E
:105F50000E944A31C8010E94152FC8010E94202FBB
:105F6000D0CF68960FB6F894DEBF0FBECDBFDF91DD
:105F7000CF911F910F91FF90EF90DF90089564E60D
:105F800070E00E94B038CB0163E00E94311583E4D9
:105F90000C94921368EE73E00E94B038CB0163E07A
:105FA0000E94311586E50C949213CF93DF9364E63B
:105FB00070E00E94B0389B01EC0163E0C9010E94CF
:105FC00031158EE20E949213CE016AE070E00E94C9
:105FD000B038862F0E94BF1385E697E0DF91CF91FE
:105FE0000C944113DC015F96ED91FC919097EE0FBC
:105FF000FF1FE759F84F859194910C9441130B962C
:106000000E94E52E24E630E040E050E00E94C438D3
:1060100065E0C9010E94311580E30E94921380E37C
:106020000C949213FC0124E6269FC001279F900D3B
:10603000112420813181820F931F8436910510F441
:1060400084E690E091838083808191818D3A9642AD
:1060500020F08CEA96E2918380830895FC012AE087
:10606000269FC001279F900D112420813181820F2E
:10607000931F8A30910510F48AE090E09183808329
:1060800080819181893E934020F088EE93E0918356
:1060900080830895FC0128EE33E0629FC001639F76
:1060A000900D729F900D112420813181820F931FDA
:1060B00088352BE1920710F488E59BE1918380837A
:1060C000808191818133954720F080E395E791832A
:1060D00080830895FC0180819181680F791F63306E
:1060E000710518F07183608304C083E090E09183B0
:1060F000808380819181893C910520F088EC90E03B
:106100009183808308950F931F93262F443019F0B5
:106110006FEF7FEF02C061E070E0022F10E00C3003
:106120001105D8F5F801EA5BFF4F0C94053941E001
:106130000B962FC00D961F910F910C9412300F9655
:106140001F910F910C942E3044E1419622C044E1FE
:1061500043961FC045E0459602C04AEF47961F91FF
:106160000F910C945F2949961F910F910C944A301E
:1061700048EE53E04B961F910F910C9476294D9663
:106180001F910F910C946A3044E04F9602C044E096
:1061900081961F910F910C944B291F910F91089597
:1061A0001F93CF93DF93EC01162F0E947517CE013A
:1061B00009960E94CC29882311F0298501C02FEF70
:1061C000332727FD3095812F90E02817390709F4F0
:1061D00042C0412F50E04C305105E8F5FA01EE5A2B
:1061E000FF4F0C9405398B850E94891334C08D852F
:1061F0009E850E94BF2F2FC08F8598890E94D52F22
:106200002AC065E089899A891CC065E08B899C89D0
:1062100018C063E08D899E890E9431151CC065E01D
:106220008F89988D0E94481516C0898D9A8D0E947D
:10623000CA2F11C066E08B8D9C8D03C065E08D8DEB
:106240009E8D0E94511507C0CE010E94F22F03C0FF
:10625000CE010E94FF2FDF91CF911F910895CF9320
:106260000E94F40AC82F882349F080915F038111AE
:1062700002C00E94AA1F87E00E944A31C0935F03B8
:106280008C2FCF9108950E946E28709364036093C1
:106290006303089590916003981721F08093600341
:1062A0000C944331089590916003983011F40C944C
:1062B0004A31089588E00C944A319B01220F331F24
:1062C0002817390764F0681779072CF4A901481BCF
:1062D000590BCA010895181619060CF4089580E0A8
:1062E00090E00895969587958531910520F46AE0B0
:1062F00070E00C945D310E945A3180E090E0089586
:106300000F931F93CF93DF93EC01D695C795D69546
:10631000C795C93CD1052CF00E945A3180E090E02D
:106320000EC06AE070E0CE010E945D318C016AE02F
:1063300070E0CE0188970E945D31800F911FDF9140
:10634000CF911F910F91089560ED77E00E94B038D2
:106350006AE070E00C945D316AE070E00E94B03851
:10636000CB016D38710520F464E170E00C945D316F
:106370000E945A3180E090E008956AE070E00E9447
:10638000B0389B01CB0168E270E00E94B038283B36
:10639000314020F464E170E00C945D310E945A3188
:1063A00080E090E008956AE070E00E94B0389B01C0
:1063B000CB0168E270E00E94B0382135310520F44D
:1063C00064E170E00C945D310E945A3180E090E00D
:1063D00008956AE070E00E94B0389B01CB0168E24A
:1063E00070E00E94B038283B314020F464E170E056
:1063F0000C945D310E945A3180E090E00895409104
:10640000600350E04830510598F4FA01E25AFF4F1A
:106410000C9405390C9472310C94A4310C94AC3169
:106420000C94BD310C9480310C94D3310C94E9312F
:1064300080E090E008950E946E28209163033091DF
:106440006403CB01821B930B0E94FF3120916103F7
:10645000309162038217930731F090936203809327
:1064600061030C9419050895CF93DF931F92CDB764
:10647000DEB7E0919D04F0919E04309711F4E1EABB
:10648000F4E0CE0101962EEB8E179F0710F02193BA
:10649000FBCF0F90DF91CF910895CF93DF9300D082
:1064A000CDB7DEB720919D0430919E0421153105B2
:1064B00011F421EA34E0CE010196821B930B0F9078
:1064C0000F90DF91CF910895CF93DF931F92CDB7B7
:1064D000DEB720919D0430919E042115310511F401
:1064E00021EA34E0F901AE014F5F5F4FCF01821B1B
:1064F000930B4E175F0728F060816E3B11F43196C5
:10650000F5CF0F90DF91CF91089587E493E00E943B
:10651000E52EAB01BC018EE693E00C9485358091AD
:106520006900813059F480915B0390915C03892B61
:1065300029F00E94853282E0809369000895CF930C
:10654000C82F682F8EE693E00E944B379091650329
:106550009C2790936503CF9108958BE30C949F3211
:10656000CF93DF93EC018991882319F00E949F3229
:10657000FACFDF91CF9108950F931F93CF93DF93BD
:10658000CDB7DEB72B970FB6F894DEBF0FBECDBFE9
:106590008E010F5F1F4F1A87098727E02B87AC01F9
:1065A000BE01655F7F4FCE0109960E945A12C80155
:1065B0000E94B0322B960FB6F894DEBF0FBECDBF4F
:1065C000DF91CF911F910F910895CF93DF93EC014D
:1065D0001092650384E20E949F32CE010E94BC3279
:1065E0000E94AD328091670090E00E94BC320E9410
:1065F000AD3260916603709167038091680390915A
:10660000690328EE33E040E050E00E94C438C9013D
:106610000E94BC328EE20E949F32609166037091AC
:106620006703809168039091690324E630E040E0BD
:1066300050E00E94C438CA01B9012AE030E040E0CD
:1066400050E00E94C438CB010E94BC32DF91CF9150
:106650000C94AD328DE00E949F328AE00C949F3200
:106660008091650390E00E94BC320C942A33CF9352
:10667000DF9381E090E00E94E532C5E3D8E0F8E0E6
:10668000C334DF0751F0FE0184910E9487080E9405
:10669000BC320E94AD322196F2CFC0E08C2F0E9416
:1066A00083260E94BC320E94AD32CF5FC630B1F764
:1066B0000E948D260E94BC320E94AD320E94932619
:1066C0000E94BC320E94AD32DF91CF910C943033E6
:1066D000CF93DF93D82F82E090E00E94E532C0E0B4
:1066E0008C2FDD2319F00E947E0802C00E948708CB
:1066F0000E94BC320E94AD32CF5FC43289F78091D4
:10670000630290E00E94BC320E94AD320E941A06E1
:106710008091D7029091D8020E94BC320E94AD3283
:10672000DF91CF910C94303383E090E00E94E5320A
:106730000E9464320E94BC320E94AD320E944D32EF
:106740000E94BC320E94AD320C943033CF93DF9361
:10675000C0915B03D0915C030E943733C230D105F6
:106760006CF081E0C430D1050CF480E00E94683305
:10677000229721F0DF91CF910C949433DF91CF9148
:1067800008950F931F9380916900813051F10E9409
:10679000D32820916900223051F460936A037093EA
:1067A0006B0380936C0390936D03109269000091CA
:1067B0006A0310916B0320916C0330916D03DC012F
:1067C000CB01801B910BA20BB30B809366039093BC
:1067D0006703A0936803B09369031F910F910C9412
:1067E000A6331F910F9108950F931F93CF93DF93BB
:1067F0001F92CDB7DEB78A0169830E949F326981FB
:10680000862F90E00E94BC328DE30E949F32C80127
:106810000E94BC320F90DF91CF911F910F910C9489
:106820002A331F93CF93DF9300D000D0CDB7DEB7CC
:106830008FEC90E00E94B0320E942A3347E050E093
:1068400060E085E40E94F43341E050E061E085E4DB
:106850000E94F43342E050E062E085E40E94F433A9
:1068600010E040E0612FCE0101960E94AA08498104
:106870005A81612F81E60E94F4334B815C81612F44
:1068800082E70E94F43341E0612FCE0101960E941D
:10689000AA0849815A81612F81E40E94F4334B8117
:1068A0005C81612F82E50E94F4331F5F1131C9F6CC
:1068B0000F900F900F900F90DF91CF911F9108953F
:1068C0008EE693E00E94CC348EE693E00E94FA3587
:1068D00060E08AE00C94DB3780916900813029F018
:1068E0000E94603481E08093690008950E9485329F
:1068F0000E9411340E942A330E9411340E942A33CC
:106900000C946034FC0124853585F901F395808170
:106910009181F901EE5FFE4F20813181821B930B43
:1069200099270895FC0184859585FC01F3954081A4
:106930005181FC01EE5FFE4F2081318142175307E8
:1069400041F00190F081E02DE80FF91F808190E087
:1069500008958FEF9FEF0895FC0184859585FC01D4
:10696000F39540815181FC01EE5FFE4F2081318122
:106970004217530771F0A081B181A80FB91F8C9104
:10698000208131812F5F3F4F33273183208390E077
:1069900008958FEF9FEF0895FC0181A1882329F0CE
:1069A000A489B5898C9186FFFBCF11A20895CF935E
:1069B000DF93FC0126853785D901B3958D919C9194
:1069C000119701969927E901CE5FDE4F48815981E1
:1069D00084179507D9F30D90BC91A02DA20FB31F7A
:1069E0006C93A685B785B39511969C938E93A689D3
:1069F000B7892C9181E090E0078C02C0880F991F25
:106A00000A94E2F7282B2C9381E081A30488F5896E
:106A1000E02D80818064808381E090E0DF91CF91E0
:106A2000089508951F920F920FB60F9211242F937D
:106A30003F934F938F939F93EF93FF935A991AC06D
:106A40004CB18091900490919104019699272091E6
:106A50009204309193048217930769F0E0919004B7
:106A6000F0919104E057FC4F408390939104809300
:106A7000900401C08CB1FF91EF919F918F914F9144
:106A80003F912F910F900FBE0F901F9018958EE69B
:106A900093E00E948234892B11F00C9411350895F3
:106AA0001F920F920FB60F9211242F933F938F9343
:106AB0009F93EF93FF9320919004309191048091E4
:106AC0009204909193042817390711F4559812C035
:106AD000E0919204F0919304E057FC4F2081809163
:106AE0009204909193040196992790939304809334
:106AF00092042CB9FF91EF919F918F913F912F912B
:106B00000F900FBE0F901F901895CF92DF92EF92CB
:106B1000FF92CF93DF93EC016A017B01411581EE77
:106B2000580761057105F9F0EC89FD8981E090E075
:106B300008A002C0880F991F0A94E2F7808360E0E2
:106B400079E08DE390E0A70196010E94C4382150BE
:106B500031094109510956954795379527952115D2
:106B600080E1380798F0EC89FD89108260E874E8CC
:106B70008EE190E0A70196010E94C43821503109AE
:106B8000410951095695479537952795E889F9891F
:106B90003083EA89FB89208319A2EE89FF8940812D
:106BA00081E090E09C010D8C02C0220F331F0A94FB
:106BB000E2F7422B4083EE89FF8940819C010E8CD5
:106BC00002C0220F331F0A94E2F7422B4083EE8962
:106BD000FF8920810F8C02C0880F991F0A94E2F769
:106BE000809582238083DF91CF91FF90EF90DF909B
:106BF000CF900895CF93DF93FC0186859785DC01C4
:106C0000B395EC01CE5FDE4F4D915C9111972881D9
:106C1000398142175307C1F7A689B7894C9181E0A2
:106C200090E09C01058C02C0220F331F0A94E2F70A
:106C3000209524232C93A689B7894C919C01068C1E
:106C400002C0220F331F0A94E2F7209524232C93CD
:106C5000A689B7892C91078C02C0880F991F0A94C6
:106C6000E2F7809582238C9384859585FC01EE5F05
:106C7000FE4F20813181FC01F39531832083DF9128
:106C8000CF910895109271031092700388EE93E0F3
:106C9000A0E0B0E08093720390937303A093740319
:106CA000B09375038AED90E090936F0380936E0329
:106CB00080E993E090937B0380937A0390937D0324
:106CC00080937C0380E490E090937F0380937E0325
:106CD00029E230E030938103209380032BE230E0FF
:106CE00030938303209382032AE230E030938503BC
:106CF0002093840390938703809386038CE290E033
:106D0000909389038093880384E080938A0383E0CF
:106D100080938B0387E080938C0385E080938D03C1
:106D200081E080938E0308950F931F93CF93DF9399
:106D300000D0CDB7DEB78C0169837A830E945339C6
:106D400069817A818617970729F0C8010E947A39EC
:106D500081E001C080E00F900F90DF91CF911F91F3
:106D60000F910895CF93DF93C82F6DE578E08CE401
:106D700098E00E942F1F67E070E080E090E00E94A2
:106D8000943681111DC0C1111BC061E070E08AE81A
:106D900090E00E94943681111BC0C11119C0D0E04F
:106DA00062E070E08CE693E00E949436811118C096
:106DB000D11116C0CC23F9F0DF91CF910C94A01F14
:106DC00089E498E00E9441130E94DD08C1E0DDCF14
:106DD00086E498E00E9441130E94FA1AD1E0E0CFC5
:106DE00083E498E00E9441130E940F2F80ED97E00A
:106DF0000E94E328DFCFDF91CF9108950E94AA3748
:106E00000E945110C7E4D5E30E943F102097E1F3A0
:106E10000E944735F9CFCF92DF92EF92FF920F9306
:106E20001F93CF93DF936C017A01EB01E60EF71EFF
:106E300000E010E0CE15DF0561F06991D601ED911B
:106E4000FC910190F081E02DC6010995080F191FF2
:106E5000F1CFC801DF91CF911F910F91FF90EF907B
:106E6000DF90CF9008956115710581F0DB010D90E1
:106E70000020E9F7AD0141505109461B570BDC01D9
:106E8000ED91FC910280F381E02D099480E090E087
:106E900008950C943337DC01ED91FC910190F08161
:106EA000E02D099480936A0008951F920F920FB607
:106EB0000F9211242F933F938F939F93AF93BF9380
:106EC0008091950490919604A0919704B0919804B4
:106ED0003091940423E0230F2D3720F40196A11D57
:106EE000B11D05C026E8230F0296A11DB11D2093F8
:106EF00094048093950490939604A0939704B09380
:106F000098048091990490919A04A0919B04B09167
:106F10009C040196A11DB11D8093990490939A043D
:106F2000A0939B04B0939C04BF91AF919F918F91CC
:106F30003F912F910F900FBE0F901F9018950197C2
:106F4000009739F0880F991F880F991F02970197B2
:106F5000F1F70895789483B7826083BF83B7816027
:106F600083BF89B7816089BF1EBC8EB582608EBD2C
:106F70008EB581608EBD8FB581608FBD85B5846013
:106F800085BD85B5806485BD329A319A309A379A2D
:106F90001AB80895843039F0853049F0833051F4BF
:106FA0008FB58F7702C08FB58F7D8FBD089585B562
:106FB0008F7D85BD0895CF93DF9390E0FC01EC5663
:106FC000F74F2491FC01EF53F74F8491882349F147
:106FD00090E0880F991FFC01EE5FF64FA591B491E8
:106FE0008850974FFC01C591D4919FB7611108C09B
:106FF000F8948C91209582238C93888182230AC0F7
:10700000623051F4F8948C91322F309583238C9315
:107010008881822B888304C0F8948C91822B8C9376
:107020009FBFDF91CF9108950F931F93CF93DF936D
:107030001F92CDB7DEB7282F30E0F901E959F74F9D
:107040008491F901EC56F74F1491F901EF53F74F82
:1070500004910023C9F0882321F069830E94CA3774
:107060006981E02FF0E0EE0FFF1FE850F74FA59188
:10707000B4919FB7F8948C91611103C0109581234E
:1070800001C0812B8C939FBF0F90DF91CF911F91F7
:107090000F910895CF93DF93282F30E0F901E9593C
:1070A000F74F8491F901EC56F74FD491F901EF5362
:1070B000F74FC491CC2391F081110E94CA37EC2F75
:1070C000F0E0EE0FFF1FE251F74FA591B4912C9124
:1070D0002D2381E090E021F480E002C080E090E088
:1070E000DF91CF910895A29FB001B39FC001A39FEC
:1070F000700D811D1124911DB29F700D811D1124F1
:10710000911D08950E947338B7FF0895821B930B59
:1071100008950E947338A59F900DB49F900DA49F71
:10712000800D911D11240895DB018F939F930E9480
:107130008938BF91AF91A29F800D911DA39F900DA3
:10714000B29F900D11240895991B79E004C0991FF6
:10715000961708F0961B881F7A95C9F780950895B1
:10716000AA1BBB1B51E107C0AA1FBB1FA617B7076D
:1071700010F0A61BB70B881F991F5A95A9F7809589
:107180009095BC01CD010895A1E21A2EAA1BBB1B4C
:10719000FD010DC0AA1FBB1FEE1FFF1FA217B307E3
:1071A000E407F50720F0A21BB30BE40BF50B661FF9
:1071B000771F881F991F1A9469F7609570958095BD
:1071C00090959B01AC01BD01CF010895052E97FB61
:1071D0001EF400940E94FD3857FD07D00E94C43869
:1071E00007FC03D04EF40C94FD3850954095309533
:1071F00021953F4F4F4F5F4F089590958095709523
:1072000061957F4F8F4F9F4F0895EE0FFF1F0590A1
:10721000F491E02D0994FB01DC0102C005900D9270
:1072200041505040D8F70895FC0105900020E9F73F
:10723000809590958E0F9F1F0895FB01DC014150B2
:10724000504048F005900D920020C9F701C01D92F2
:1072500041505040E0F70895FB01DC01415050409F
:1072600048F001900D920020C9F701C01D924150D5
:107270005040E0F70895DC01CB01FC01E199FECF1D
:1072800006C0FFBBEEBBE09A31960DB20D924150A5
:107290005040B8F70895E199FECF9FBB8EBBE09AAE
:1072A00099278DB30895A8E1B0E042E050E00C9436
:1072B0003D39DC01A40FB51F4150504048F0CB01CF
:1072C000840F951F2E910E946A3941505040D0F78B
:1072D0000895262FE199FECF9FBB8EBBE09A0197C0
:1072E0000DB2021631F02DBB0FB6F894E29AE19A76
:1072F0000FBE08950196272F0E946A390C946939B0
:04730000F894FFCF2F
:107304000000A1042000FF03E1010100004000147B
:107314000054000000010201020101010101010108
:1073240000000501010101000000000080100000C0
:1073340000006F170B3700000000751700000000F5
:10734400E417000000001D1C381B0506080705098A
:107354000905070000050700000000642E702A00DC
:10736400000000882E472A00000000D030833056E9
:107374003D302E33320000000000D7340B37823406
:06738400AC349234CC345D
:00000001FF
